:0200000480007A
:10000000B72F0000938F0F8073900F306F00400365
:100010001300000013000000130000001300000094
:100020001300000013000000130000001300000084
:100030001300000013000000130000001300000074
:100040009702000093824211739052309300000097
:10005000130100009301000013020000930200004E
:100060001303000093030000130400009304000036
:10007000130500009305000013060000930600001E
:100080001307000093070000130800009308000006
:100090001309000093090000130A0000930A0000EE
:1000A000130B0000930B0000130C0000930C0000D6
:1000B000130D0000930D0000130E0000930E0000BE
:1000C000130F0000930F000097110200938181CD60
:1000D000170502001305054F979503009385457694
:1000E00013060000EF00001A1705020013058543F0
:1000F000970502009385C54A13060000EF0080189B
:1001000017A503001305057497B503009385457380
:1001100037B6ABAB1306B6BAEF00C01617B1030083
:1001200013014172EF8010139392120093D21200C8
:100130009382D2FF638A02008322010013014100EF
:100140006F0000177300203083220100130141006B
:10015000730020301301C1FF23205100F32220340B
:10016000E3C402FC8322010013014100130141F8A2
:1001700023221100232421002326310023284100BB
:10018000232A5100232C6100232E71002320810299
:10019000232291022324A1022326B1022328C10293
:1001A000232AD102232CE102232EF1022320010570
:1001B0002322110523242105232631052328410567
:1001C000232A5105232C6105232E71052320810745
:1001D000232291072324A1072326B1072328C1073F
:1001E000232AD107232CE107232EF107732520347E
:1001F000F3251034130601006F000000731015344E
:1002000083204100032181008321C10003220101D9
:1002100083224101032381018323C10103240102BD
:1002200083244102032581028325C10203260103A1
:1002300083264103032781038327C1030328010485
:1002400083284104032981048329C104032A010569
:10025000832A4105032B8105832BC105032C01064D
:10026000832C4106032D8106832DC106032E010731
:10027000832E4107032F8107832FC1071301C10775
:10028000730020302320C5006376B50013054500B8
:100290006FF05FFF678000000000000000000000BA
:1002A000000000000000000000000000000000004E
:1002B000130101F8232011002322210023243100FF
:1002C0002326410023285100232A6100232C71009A
:1002D000232E8100232091022322A1022324B10294
:1002E0002326C1022328D102232AE102232CF10272
:1002F000232E010323201105232221052324310568
:100300002326410523285105232A6105232C710545
:10031000232E8105232091072322A1072324B1073F
:100320002326C1072328D107232AE107232CF1071D
:100330009702020083A2422223A02200F32210345B
:10034000232E5106EF00C03B170102000321C120FC
:10035000032101008322C10773901234B7220000E9
:100360009382028873A00230832001000322C1001F
:100370008322010103234101832381010324C1015D
:100380008324010203254102832581020326C10241
:100390008326010303274103832781030328C10325
:1003A000832801040329410483298104032AC10409
:1003B000832A0105032B4105832B8105032CC105ED
:1003C000832C0106032D4106832D8106032EC106D1
:1003D000832E0107032F4107832F81071301010893
:1003E00073002030970202009382C21D23A01200E6
:1003F00023A2220023A4320023A6420023A85200F5
:1004000023AA620023AC720023AE820023A09202D2
:1004100023A2A20223A4B20223A6C20223A8D202CC
:1004200023AAE20223ACF20223AE020323A01205A8
:1004300023A2220523A4320523A6420523A85205A0
:1004400023AA620523AC720523AE820523A092077E
:1004500023A2A20723A4B20723A6C20723A8D20778
:1004600023AAE20723ACF207EF60907317010200A2
:100470000321810E032101008322C10773901234EE
:10048000B72200009382028873A00230832001000B
:100490000322C1008322010103234101832381013F
:1004A0000324C10183240102032541028325810223
:1004B0000326C10283260103032741038327810307
:1004C0000328C103832801040329410483298104EB
:1004D000032AC104832A0105032B4105832B8105CF
:1004E000032CC105832C0106032D4106832D8106B3
:1004F000032EC106832E0107032F4107832F810797
:100500001301010873002030970202009382820BCE
:1005100083A0020003A1420083A1820003A2C200C3
:1005200083A2020103A3420183A3820103A4C201A7
:1005300083A4020203A5420283A5820203A6C2028B
:1005400083A6020303A7420383A7820303A8C2036F
:1005500083A8020403A9420483A9820403AAC20453
:1005600083AA020503AB420583AB820503ACC20537
:1005700083AC020603AD420683AD820603AEC2061B
:1005800083AE020703AFC20983AF82076780000012
:1005900073700430130101F823201100232221007D
:1005A000232431002326410023285100232A6100FF
:1005B000232C7100232E8100232091022322A102EB
:1005C0002324B1022326C1022328D102232AE102D7
:1005D000232CF102232E01032320110523222105C0
:1005E000232431052326410523285105232A6105AB
:1005F000232C7105232E8105232091072322A10797
:100600002324B1072326C1072328D107232AE10782
:10061000232CF1079702020083A202F423A02200F8
:10062000232E1106EF300074170102000321C1F2DE
:10063000032101008322C10773901234B722000006
:100640009382028873A00230832001000322C1003C
:100650008322010103234101832381010324C1017A
:100660008324010203254102832581020326C1025E
:100670008326010303274103832781030328C10342
:10068000832801040329410483298104032AC10426
:10069000832A0105032B4105832B8105032CC1050A
:1006A000832C0106032D4106832D8106032EC106EE
:1006B000832E0107032F4107832F810713010108B0
:1006C00073002030737004306F00000073104530E9
:1006D000678000007325403073F04330678000006E
:1006E00097070000938747FE232EB5FE2322C5FA05
:1006F000232635F82320F5F8130505F86780000058
:10070000130101FF23261100EF605046EF20501C1B
:10071000631805008320C1001301010167800000F8
:100720008320C100130101016F30C063930785006E
:100730001307F0FF2322F5002324E5002326F5000C
:100740002328F500232005006780000023280500EA
:10075000678000008327450023A2F50003A78700D8
:1007600023A4E50003A787002322B70023A4B70032
:1007700023A8A50083270500938717002320F500F1
:100780006780000003A605009307F0FF13078500AC
:100790006316F6006F008003138707008327470066
:1007A00083A60700E37AD6FE23A2F50023A4B700B0
:1007B00023A4E5002322B70023A8A5008327050072
:1007C000938717002320F5006780000003270501A9
:1007D000832747006FF05FFD0327450083268500D0
:1007E000832705012324D70003278500832645009E
:1007F0002322D70003A747006316A700032785001D
:1008000023A2E7002328050003A507001305F5FF31
:1008100023A0A70067800000130101FF23248100AB
:1008200023261100232291008327050413040500C9
:100830006398070283270500638C070C13050000EB
:100840008327840393871700232CF4028320C1009D
:10085000032481008324410013010101678000000B
:1008600093040600631A0604032585001386070017
:10087000EF50100C832784008326040403274400D0
:10088000B387D7002324F400E3EAE7FA83270400C0
:10089000130500002324F4008327840393871700A3
:1008A000232CF4028320C10003248100832441000F
:1008B00013010101678000000325C50013860700AE
:1008C000EF501007032704048327C4008326040085
:1008D0003307E040B387E7002326F40063F8D7002E
:1008E000832744003387E7002326E4009307200092
:1008F000E396F4F483278403E38207F483278403D5
:10090000130500009387F7FF232CF4026FF05FF3C9
:1009100003254500EF30506C232204006FF05FF296
:10092000130101FE232E1100232C8100232A9100A4
:10093000032445052326A100630E04020327840334
:100940008327C4036366F700737004306F000000F0
:1009500003278403930400006362F7028320C1012C
:100960000324810113850400832441011301010242
:1009700067800000737004306F000000138605006C
:10098000130504009305C100EFF01FE90327840459
:100990009307F0FF93040500630AF700832784049C
:1009A000938717002324F4046FF05FFB832744022E
:1009B000E38607FA13054402EF30101EE30005FA40
:1009C000930410006FF09FF9032605049387050038
:1009D000630406028325C50003274500B385C500CF
:1009E0002326B50063E6E500832505002326B50030
:1009F000138507006F50C07367800000130101FD6D
:100A000023248102232611021304050023229102CC
:100A100023202103232E3101232C4101232A5101BC
:100A2000EF30906883278404635CF004130A440267
:100A30009309F0FF1309100083244405638E04001A
:100A400003A7840383A7C403232681006368F70AEE
:100A5000737004306F000000832744026382070232
:100A600013050A00EF3050136314050C8327840428
:100A70009387F7FF2324F40483278404E34EF0FADA
:100A80009307F0FF2324F404EF305065EF30D0617A
:100A900083274404635CF002832704016388070210
:100AA0009304040113850400EF30100F631605084A
:100AB000832744049387F7FF2322F4048327440405
:100AC0006356F00083270401E39E07FC9307F0FFC1
:100AD0002322F404EF3090608320C10203248102BA
:100AE00083244102032901028329C101032A8101D0
:100AF000832A4101130101036780000003A78403D7
:100B0000E376F7F6130600009305C1001385040091
:100B1000EFF09FD083A78404930A05006382370314
:100B200083A784049387170023A4F404E3902AF591
:100B3000EF30D0336FF09FF3EF3050336FF05FF74B
:100B400083A74402E38407FE13854402EF30D004F8
:100B5000E30E05FC6FF0DFFD630A0508130101FEDB
:100B6000232C810013040500232E1100232A910059
:100B7000232821012326310113890500EF30D052AB
:100B8000832404048325C4038329040013850400FB
:100B9000EF7090461307F0FF232C0402B307954033
:100BA000B387F9003385A9002322E4042322A4009B
:100BB000232434012326F4002324E404631C0902C3
:100BC0008327040163920704EF3050518320C10151
:100BD0000324810183244101032901018329C100E8
:100BE00013051000130101026780000073700430C8
:100BF0006F00000013050401EFF05FB3130544021A
:100C0000EFF0DFB26FF05FFC13050401EF30C07846
:100C100093071000E31AF5FAEFF09F976FF0DFFAF1
:100C200063160500737004306F000000130101FEAD
:100C3000232A91002328210123263101232E11008C
:100C4000232C8100930405001389050093090600F5
:100C50006382050AEF70503A13059505EF50C02CDA
:100C6000130405006300050A930785052320F5009A
:100C7000232E940223202405EF3010438324040400
:100C80008325C4030329040013850400EF70D036C4
:100C90009306F0FF232C0402B30795403307A90005
:100CA000B307F9002322D4042322E4002326F4000E
:100CB0002324D4041305040123242401EFF01FA7E7
:100CC00013054402EFF09FA6EF305041230834058E
:100CD000232A0404130504008320C1010324810195
:100CE00083244101032901018329C1001301010269
:100CF0006780000013058005EF50002313040500F2
:100D000063160500737004306F0000002320840018
:100D10006FF01FF6130101FD2322910293040500D9
:100D20001305800523248102232611022320210399
:100D3000232E3101232C4101EF50001F1304050025
:100D400063080506232C05029307F0FF2322F50410
:100D500013071000130A05012324F40413050A00E5
:100D6000232EE40223220400232004002324040071
:100D7000232604002320040423089404232A0404C3
:100D8000EFF0DF9A1309440213050900EFF01F9AF0
:100D90008327040423220100638E0702737004304A
:100DA0006F00000013050400EFF05FC5EF20C0578F
:100DB000130504008320C10203248102832441021D
:100DC000032901028329C101032A810113010103BF
:100DD00067800000EF30900D631605008327410007
:100DE00063980710EF30502C032784038327C40334
:100DF000930400009309F0FF6362F7088327410022
:100E0000638E070A6396040013058100EF30807338
:100E1000EF30D02CEF20C01DEF3010298327440481
:100E200063943701232204048327840463943701E5
:100E300023240404EF30902A930541001305810018
:100E4000EF304073E31005F6EF30102603278403DC
:100E50008327C4036308F706EF3050281305040006
:100E6000EFF0DFB9EF20404C93041000EF30D023B7
:100E7000032784038327C403E372F7F803260404DB
:100E8000631C060683270400638A070A1305000013
:100E9000832784030327440593871700232CF40238
:100EA000630607089305000013050400EFF05FA731
:100EB000930710006314F500EFF08FEDEF30102270
:100EC0006FF01FEFEF3090218325410013050A00DA
:100ED000EF30801F13050400EFF05FB2EF20C04435
:100EE000E31405F8EFF0CFEA930410006FF01FF859
:100EF000737004306F000000032584009305000028
:100F0000EF50002383278400832604040327440032
:100F1000B387D7002324F400E3EAE7F6832704002D
:100F2000130500002324F4006FF09FF6832744028A
:100F3000639E0700E30405F86FF01FF803254400E3
:100F4000EF309009232204006FF09FF4130509008D
:100F5000EF30804493071000E312F5F66FF0DFF5F1
:100F600063160500737004306F0000006376B500EF
:100F7000737004306F000000130101FF232481000F
:100F8000130620001384050093050000232611009A
:100F9000EFF01FC9630C0500232C85028320C100DC
:100FA0000324810013010101678000007370043085
:100FB0006F000000130101FC232E1102232C81027B
:100FC000232A9102232821032326310323244103CA
:100FD00023225103232061032326C1006304051645
:100FE000638A051493072000639CF6000327C5035A
:100FF000930710006306F700737004306F00000061
:10100000938406001389050013040500EF30006A7D
:10101000631A05008327C1006386070073700430DC
:101020006F000000EF305008032784038327C403B8
:1010300093090000130B2000130AF0FF930A040128
:101040006364F708638464118327C100638C071C01
:101050006396090013058101EF30C04EEF30100890
:10106000EF101079EF305004832744046394470154
:101070002322040483278404639447012324040463
:10108000EF30D0059305C10013058101EF30804E8C
:1010900063100518EF305001032784038327C4032E
:1010A0006304F706EF30900313050400EFF01F957B
:1010B000EF20802793091000EF30007F032784037F
:1010C0008327C403E370F7F80326040463040608C7
:1010D000639004160325840093050900EF50400532
:1010E000832784008326040403274400B387D700A2
:1010F0002324F40063E4E7068327040013050000BB
:101100002324F4006F00C005EF30407D8325C1002B
:1011100013850A00EF20507B13050400EFF01F8EAB
:10112000EF208020E31805F8EFF08FC69309100038
:101130006FF09FF883270504E38607EA7370043095
:101140006F000000737004306F0000000326040479
:101150006314060683270400638C07101305000040
:10116000832784030327440593871700232CF40265
:101170006306070E9385040013050400EFF04FFA91
:10118000930710006302F50EEF3040751305100051
:101190008320C10303248103832441030329010322
:1011A0008329C102032A8102832A4102032B0102FF
:1011B00013010104678000000325C40093050900A2
:1011C000EF401077832704040327C400832604001C
:1011D000B307F0403307F7002326E400637CD70011
:1011E00003274400B307F7002326F40093072000E9
:1011F000E396F4F683278403E38207F683278403C8
:10120000130500009387F7FF232CF4026FF05FF5BE
:1012100013050400EFF08FFEEF200011130500000E
:101220006FF01FF7EF30806B130500006FF05FF673
:101230000325C40093050900EF40906F8327040441
:101240000327C40083260400B307F0403307F700E8
:101250002326E400E37CD7F86FF09FF8832744024D
:1012600063900702E30205F2EFF08FB26FF0DFF157
:1012700003254400EF304056232204006FF05FEE58
:1012800013054402EF30401193071000E31EF5EE02
:101290006FF09FFD63040504130101FF2324810007
:1012A0002322910023261100232021010329450038
:1012B00013040500EF30803E930400006304A9028C
:1012C0008320C10003248100138504000329010049
:1012D0008324410013010101678000007370043012
:1012E0006F0000008327C400930410009387F7FF6A
:1012F0002326F400E39607FC930600001306000083
:101300009305000013050400EFF0DFCA6FF05FFBE8
:101310006302050A63880508130101FE232C81007E
:10132000232A91002328210123244101232E110087
:101330002326310193072000938406001309060039
:10134000138A050013040500639CF6000327C503F8
:10135000930710006302F70A737004306F000000F7
:10136000EFF04FB7032784038327C40393090500D5
:101370006366F7049304000013850900EFF00FB5CE
:101380008320C10103248101138504000329010185
:10139000832441018329C100032A81001301010232
:1013A0006780000083270504E38807F67370043024
:1013B0006F000000737004306F0000000326040407
:1013C000631E060C832704006388071283278403A7
:1013D0001307F0FF93871700232CF402832784045C
:1013E0006388E70E83278404930410009387170013
:1013F0002324F4046FF05FF8EFF0CFAD03278403EC
:101400008327C403930905006360F70603260404D9
:10141000E30A06FA0325C40093050A00EF40505181
:10142000832704040327C40083260400B307F04085
:101430003307F7002326E4006378D700032744002E
:10144000B307F7002326F40093072000E390F4F895
:1014500083278403E38C07F6832784039387F7FFAE
:10146000232CF4026FF09FF603260404E30C06F429
:101470000325C40093050A00EF40904B8327040422
:101480000327C40083260400B307F0403307F700A6
:101490002326E400E364D7FA6FF09FFBE39C04F695
:1014A0000325840093050A00EF40904883278400B9
:1014B0008326040403274400B387D7002324F400C1
:1014C000E3E6E7F0832704002324F4006FF01FF025
:1014D00083274405638A07029385040013050400EB
:1014E000EFF00FC493041000E31895E8E30609E851
:1014F000232099006FF05FE803254400EF30C02DF2
:10150000232204006FF09FEC832744029304100011
:10151000E38407E613054402EF201068E31805FC96
:101520006FF09FE56302050A8327050463860700C1
:10153000737004306F00000083270500638A07087A
:10154000130101FE232C8100232A910013040500BE
:101550002328210123263101232E110013890500A0
:10156000EFF04F97032784038327C40393090500F3
:10157000930400006376F702832784031307F0FFC8
:1015800093871700232CF40283278404638AE704DB
:101590008327840493041000938717002324F40402
:1015A00013850900EFF08F928320C101032481018C
:1015B0001385040003290101832441018329C1000B
:1015C0001301010267800000737004306F00000097
:1015D00083274500E38607F6737004306F00000030
:1015E0008327440563800702930500001305040068
:1015F000EFF00FB3930710006300F502930410009F
:101600006FF01FFA83274402E38A07FE13054402A2
:10161000EF209058E30405FEE30209FE9307100053
:101620002320F9006FF09FFD130101FC232E11020E
:10163000232C8102232A910223282103232631030C
:10164000232441032326C100630005166386051485
:10165000938906001389050013040500EF30000587
:10166000631A05008327C100638607007370043086
:101670006F000000EF30402383278403639E070A36
:101680008327C1006388071813058101EF20906B41
:101690009304F0FF130A44026F008002EF3000242D
:1016A00013050400EFF08FB5EF101048EF30C01FA6
:1016B00083278403639207088327C100638C071480
:1016C000EF30C021EF10D012EF30001E832744040A
:1016D000639497002322040483278404639497006F
:1016E00023240404EF30801F9305C10013058101FA
:1016F000EF20506863160510EF30001B832784032A
:10170000E39E07F8EF30801D832704006386070AF5
:101710008325C10013050A00EF20101B13050400E8
:10172000EFF0CFADEF10504063040508EF30C01765
:1017300083278403E38207F8930509001305040057
:101740008324C400EFF04FA8639209088327840321
:10175000032704009387F7FF232CF4026316070086
:10176000EF30001F2322A4008327040163900708A1
:10177000EF30C016130510008320C103032481033A
:1017800083244103032901038329C102032A81021F
:10179000130101046780000083270504E38A07EA38
:1017A000737004306F000000737004306F0000002D
:1017B000EFE01FDE6FF09FF7EF30000F03254400CE
:1017C000EF209071EF3080116FF09FF48327440277
:1017D00023269400E38E07F813054402EF20D03B44
:1017E000E30805F8EFE0DFDA6FF09FF81305040176
:1017F000EF20903A93071000E31CF5F66FF09FFE80
:1018000013050400EFF08F9FEF1010321305000056
:101810006FF09FF6EF30800C130500006FF0DFF5DE
:1018200063000506130101FF232481002320210109
:1018300023261100232291008324450013890500EB
:1018400013040500EF2090656380A4049306000054
:10185000130609009305000013050400EFF0DFDC18
:1018600093071000630CF5028320C100032481005C
:101870008324410003290100130101016780000056
:10188000737004306F0000008327C400130510003C
:10189000938717002326F4006FF01FFD8327C400F1
:1018A000938717002326F4006FF01FFC63080506DA
:1018B0006386050C130101FE232C8100232A91006D
:1018C000232821012326310123244101130405008B
:1018D000232E11001309060093890500EFE09FDF16
:1018E00083278403130A050093040000639C070206
:1018F00013050A00EFE09FDD8320C101032481016D
:101900001385040003290101832441018329C100B7
:10191000032A810013010102678000007370043004
:101920006F00000003260404630406028325C4003C
:1019300083274400B385C5002326B40063E6F50081
:10194000832504002326B40013850900EF40407E60
:10195000832784031307F0FF9387F7FF232CF402F8
:10196000832744046384E70283274404930410001C
:10197000938717002322F4046FF09FF78327050451
:10198000E38A07F2737004306F00000083270401BC
:1019900063960700930410006FF09FF51305040190
:1019A000EF20901FE30805FEE30609FE93071000F1
:1019B0002320F9006FF01FFE630605088327050446
:1019C000638A050863840708130101FE232C810044
:1019D000232A910023282101232441011304050017
:1019E000232E110023263101138A0500EFE09FCE3C
:1019F000832784031309050093040000638E070006
:101A00008329C40093050A0013050400EFE0DFFBFF
:101A1000930410002326340113050900EFE01FCBC7
:101A20008320C101032481011385040003290101DE
:101A3000832441018329C100032A8100130101028B
:101A400067800000737004306F0000007370043012
:101A50006F000000E38C07FE737004306F0000001D
:101A600063160500737004306F000000130101FF5E
:101A7000232481001304050023261100EF20D062E7
:101A800003248403EF2090658320C1001305040024
:101A90000324810013010101678000006316050023
:101AA000737004306F000000130101FF2326110042
:101AB0002324810013040500EF20105F8327840393
:101AC0000324C4033304F440EF20506113050400E1
:101AD0008320C100032481001301010167800000FD
:101AE00063060500032585036780000073700430DA
:101AF0006F0000006308050497870300938787D071
:101B000003A747006304E50403A7C7006302E508D1
:101B100003A74701630AE50603A7C7016302E506B9
:101B200003A74702630AE50403A7C7026302E504AB
:101B300003A74703630AE50203A7C7036302E5029D
:101B40006F408056737004306F0000001307000070
:101B500013173700B387E70023A007006F40C05476
:101B6000130770006FF0DFFE130760006FF05FFE79
:101B7000130750006FF0DFFD130740006FF05FFDAB
:101B8000130730006FF0DFFC130720006FF05FFCDD
:101B9000130710006FF0DFFB0325C504678000000A
:101BA0002326B50467800000034505056780000013
:101BB00063080500032585031335150067800000C1
:101BC000737004306F000000630C050083278503E9
:101BD0000325C5033305F540133515006780000064
:101BE000737004306F00000097870300938787C1EC
:101BF00003A707006300070403A78700630807041F
:101C000003A707016308070403A787016308070404
:101C100003A707026308070403A7870263080704F2
:101C200003A70703630C070403A7870363040704E0
:101C3000678000001307000013173700B387E70021
:101C400023A0B70023A2A70067800000130710009D
:101C50006FF09FFE130720006FF01FFE1307300088
:101C60006FF09FFD130740006FF01FFD130750003A
:101C70006FF09FFC130770006FF01FFC13076000EC
:101C80006FF09FFB978703009387C7B703A74700B1
:101C90006300E50403A7C7006306E50403A7470143
:101CA0006306E50403A7C7016306E50403A747022B
:101CB0006306E50403A7C7026306E50403A7470319
:101CC000630AE50403A7C7036302A7046780000053
:101CD0001307000013173700B387E70023A007009E
:101CE00067800000130710006FF0DFFE130720006D
:101CF0006FF05FFE130730006FF0DFFD1307400049
:101D00006FF05FFD130750006FF0DFFC13077000EA
:101D10006FF05FFC130760006FF0DFFB130101FD44
:101D2000232481022322910223202103130405008E
:101D300023261102232E3101232C4101232A510194
:101D40009384050013090600EF201036032744048E
:101D50009307F0FF6314F70023220404032784048D
:101D60009307F0FF6314F70023240404EF201037D7
:101D700083278403639A07001306090093850400F0
:101D800013054402EF208050EF2010328327840493
:101D9000635CF004130A44029309F0FF1309100076
:101DA00083244405638E040003A7840383A7C4032C
:101DB000232681006368F70A737004306F00000007
:101DC000832744026382070213050A00EF20C05CE8
:101DD0006314050C832784049387F7FF2324F404FA
:101DE00083278404E34EF0FA9307F0FF2324F404DE
:101DF000EF20D02EEF20502B83274404635CF002A9
:101E000083270401638807029304040113850400F7
:101E1000EF20805863160508832744049387F7FF53
:101E20002322F404832744046356F000832704012B
:101E3000E39E07FC9307F0FF2322F404EF20102A0F
:101E40008320C10203248102832441020329010269
:101E50008329C101032A8101832A4101130101035E
:101E60006780000003A78403E376F7F613060000FB
:101E70009305C10013850400EFE01F9A83A7840433
:101E8000930A05006382370383A7840493871700AE
:101E900023A4F404E3902AF5EF20407D6FF09FF334
:101EA000EF20C07C6FF05FF783A74402E38407FE56
:101EB00013854402EF20404EE30E05FC6FF0DFFD7A
:101EC00063160500737004306F000000130101FFFA
:101ED0002322910093040500131525001305950591
:101EE000232481002326110023202101EF40C00379
:101EF0001304050063080508930785052320F500F2
:101F0000930740002320F504232E9502EF20D019DB
:101F1000832404048325C4030329040013850400D7
:101F2000EF60900D9306F0FF232C0402B307954059
:101F30003307A900B307F9002322D4042322E400C5
:101F40002326F4002324D4041305040123242401AC
:101F5000EFE0CFFD13054402EFE04FFDEF20101836
:101F600023080404232A0404130504008320C10069
:101F7000032481008324410003290100130101018E
:101F800067800000737004306F000000130101FFD0
:101F90002324810023229100232021011304050022
:101FA0002326110013890500EF2010108327440514
:101FB0009304000063820702EF2050128320C100C7
:101FC00003248100138504000329010083244100B8
:101FD000130101016780000083278403930400003C
:101FE000E39C07FC232A2405930410006FF0DFFC18
:101FF000832745056388B700930700001385070012
:10200000678000000327850393070000E31807FE9D
:10201000130101FF2324810013040500232611006E
:10202000EF209008232A0404EF20500B8320C100E6
:102030000324810093071000138507001301010199
:1020400067800000130101FE13860500930600005F
:102050009305C100232E110023260100EFF0CFDCF1
:102060008320C1010325C100130101026780000024
:10207000130101FE232E1100232C8100232A91003D
:1020800023260100630C050213040500EFE08FE432
:1020900083278403930405006396070213850400D5
:1020A000EFE0CFE28320C101032481010325C100B9
:1020B0008324410113010102678000007370043022
:1020C0006F00000003260404630406028325C40095
:1020D00083274400B385C5002326B40063E6F500DA
:1020E000832504002326B4001305C100EF404004FB
:1020F000832784031307F0FF9387F7FF232CF40251
:1021000083274404638AE7008327440493871700E6
:102110002322F4046FF09FF883270401E38007F87B
:1021200013050401EF2040276FF05FF763020504F9
:10213000130101FD232E3101232C4101232611021D
:10214000138A0700232481022322910223202103E2
:10215000232A51012328610123267101930790004E
:102160009309070063FAE700737004306F00000002
:10217000737004306F000000130B0500938405009A
:1021800013090600938B0600930A08006302082CCB
:1021900013050006EF305059130405006302052AA9
:1021A0001319290023285503130609009305500A23
:1021B00013850A00EF40C00903C704008327040306
:1021C0001309C9FF230AE40203C704003389270166
:1021D0001379C9FF6306070E83C71400A30AF4022C
:1021E00083C71400638E070C83C72400230BF402FB
:1021F00083C724006386070C83C73400A30BF40253
:1022000083C73400638E070A83C74400230CF4029B
:1022100083C744006386070A83C75400A30CF402F3
:1022200083C75400638E070883C76400230DF4023C
:1022300083C764006386070883C77400A30DF40294
:1022400083C77400638E070683C78400230EF402DD
:1022500083C784006386070683C79400A30EF40235
:1022600083C79400638E070483C7A400230FF4027E
:1022700083C7A4006386070483C7B400A30FF402D6
:1022800083C7B400638E070283C7C4002300F4042D
:1022900083C7C4006386070283C7D400A300F40485
:1022A00083C7D400638E070083C7E4002301F404CE
:1022B00083C7E4006386070083C7F400A301F40426
:1022C000930A440013850A00A3010404232634035F
:1022D00023283405232A0404EFE04FC713058401A3
:1022E000EFE0CFC69307A000B3873741232C040447
:1022F00023288400232CF4002322840223220404B4
:10230000232E040413860B0093050B00130509000C
:10231000EFE00FBD2320A40063040A0023208A00FD
:102320007370043017E9010013094921832709005C
:1023300097E4010093844422638C070003A7040000
:1023400083A7040083274704938717002322F704F9
:1023500017E701001307471F83270700938717001C
:1023600097E6010023A2F61E83A70400638E070EE2
:102370008327090017EB0100130B8B2C639C0700CC
:1023800083A7040083A7C70263E6F90097E701006B
:1023900023A4871C97E701009387471983A70700A9
:1023A00017E701001307C7190325C4020327070015
:1023B0009387170097E6010023AAF6162324F40456
:1023C0006376A70097E7010023ACA71693054001A9
:1023D000EF60804293850A003305AB00EFE08FB7D2
:1023E000832709006388070083A7040083A74704A5
:1023F000639C07088327090013041000638A070001
:1024000083A7040083A7C70263F43701EFE04F9866
:10241000130504008320C1020324810283244102A6
:10242000032901028329C101032A8101832A410171
:10243000032B0101832BC1001301010367800000FE
:1024400013850A00EF3050461304F0FF6FF05FFC75
:1024500013152600EF30502D930A0500E31A05D21C
:102460001304F0FF6FF0DFFA97E7010023A6870E51
:102470000327070093071000630AF70217EB010018
:10248000130B0B1C6FF01FF103A7040083A60400BD
:10249000832747049387F7FF2322F70483A7460483
:1024A000E39A07F4736004306FF0DFF4130A00005E
:1024B00017EB0100130BCB18930BA00013050A00B8
:1024C00093054001EF604033130A1A003305AB0057
:1024D000EFE0CFA5E3147AFF97EB0100938BCB22BB
:1024E00013850B00EFE08FA417EA0100130A0A23FB
:1024F00013050A00EFE08FA317E50100130545233C
:10250000EFE0CFA217E501001305C523EFE00FA20E
:1025100017E5010013054524EFE04FA197E70100FF
:1025200023AA770397E7010023A447036FF09FE6F0
:10253000130101FF2324810023261100232291008F
:1025400023202101130405007370043097E4010077
:102550009384C4FE83A70400639E071063180400DD
:1025600097E70100938747FF03A40700130944007E
:1025700013050900EFE04FA6832784026386070056
:1025800013058401EFE04FA59305090017E501004D
:102590001305451BEFE00F9C97E70100938707FBAE
:1025A00003A7070097E70100938747F883A7070071
:1025B0001307170097E6010023AAE6F803A7040013
:1025C0009387170097E6010023A2F6F6630C070035
:1025D00097E70100938747F803A7070003274704FD
:1025E000631C070E83A70400638A070697E70100B0
:1025F000938787F603A70700630287107370043080
:1026000003A704006318070817E70100130787F4FE
:102610008326070083A606006392060A1307F0FFCD
:1026200097E6010023A2E6F003A70400630807026F
:1026300003A70700032747046302070203A7070055
:1026400083A60700832747049387F7FF2322F70415
:1026500083A7460463940700736004308320C1009D
:102660000324810083244100032901001301010197
:102670006780000097E70100938707EE03A7070034
:1026800083A7070083274704938717002322F704B3
:102690006FF0DFEC83A6070003A7070003A746043B
:1026A0001307170023A2E60417E70100130787EAC0
:1026B0008326070083A60600E38206F603270700A9
:1026C0000327C7000327C7000327470097E6010039
:1026D00023ACE6E46FF05FF503A7070083A60700CD
:1026E000832747049387F7FF2322F70483A7460431
:1026F000E39A07EE736004306FF0DFEE97E70100B6
:10270000938747E283A7070063860700737004304E
:102710006F000000032481008320C1008324410056
:1027200003290100130101016FD09FE66304050C2A
:1027300017E70100130747E283260700930700000D
:102740006386A60A130101FF2326110023248100BA
:10275000232291007370043097E60100938606DE11
:1027600083A70600638C0700032607008327070062
:1027700083274604938717002322F60483A70600C5
:10278000930405000324450163880700832707009D
:1027900083A747046394070697E70100938787DBC5
:1027A00083A70700638C870697E70100938747DAC2
:1027B00083A707006384870697E701009387C7F91B
:1027C0006306F40497E701009387C7F7630CF402EC
:1027D000930710008320C10003248100832441005B
:1027E00013850700130101016780000013850700AE
:1027F00067800000737004306F000000EF60C01548
:102800006FF09FF9930740006FF0DFFC83A784020D
:1028100093B71700938727006FF0DFFB9307200023
:102820006FF05FFB7370043097E70100938707D167
:1028300003A70700631607026304050483A70700C4
:102840000325C502638C070097E701009387C7D073
:1028500003A7070003274704631C070267800000E3
:1028600017E70100130747CF832607000327070058
:1028700003A746041307170023A2E604E31005FC90
:1028800017E70100130747CD032507006FF01FFB73
:1028900003A7070083A60700832747049387F7FF52
:1028A0002322F70483A74604E39A07FA73600430EF
:1028B00067800000130101FF232481001304050039
:1028C00023261100EFD01FE16318040097E70100F1
:1028D000938787C803A407000324C402EFD01FDF37
:1028E0008320C100130504000324810013010101AA
:1028F000678000009307900063F6B70073700430A0
:102900006F000000130101FE232C8100232E110013
:10291000232A910023282101232631012324410168
:10292000130405007370043017E90100130909C18D
:1029300083270900639207106300041283270405AC
:10294000638EF50A17E70100130707C163F0B702AA
:1029500083260700638E8612032707008324C7029D
:10296000B3B4950093C414006F00000183240700E2
:10297000B384844093B414000327C4026386E70E33
:10298000832784012328B40463C807009307A000A9
:10299000B385B740232CB40093172700B387E70013
:1029A0000327440197E90100938989C99397270078
:1029B000B387F9006310F704130A440013050A00F3
:1029C000EFD09FE197E70100938787B70325C40203
:1029D00083A7070063F6A70097E7010023A2A7B625
:1029E00093054001EF50506193050A003385A9001B
:1029F000EFD05FD663840400EFD09FB9832709002E
:102A0000638C070097E70100938707B583A707004A
:102A100083A74704639E07048320C1010324810127
:102A200083244101032901018329C100032A810074
:102A3000130101026780000097E701009387C7B187
:102A400003A7070083A7070083274704938717007E
:102A50002322F704E31404EE97E701009387C7AF3E
:102A600003A407006FF09FED2326B4026FF05FF11F
:102A7000032481018320C101832441010329010131
:102A80008329C100032A8100130101026F50D06C19
:102A9000930400006FF05FEE630A0508130101FE66
:102AA000232A910097E40100938404AB83A70400D8
:102AB000232E1100232C81002328210123263101FC
:102AC0006388A7047370043017E90100130909A78C
:102AD00083270900638C070003A7040083A7040071
:102AE00083274704938717002322F7040327450110
:102AF00097E70100938747C6630EF7028327090013
:102B00006388070083A7040083A74704639E070820
:102B10008320C10103248101832441010329010190
:102B20008329C10013010102678000007370043023
:102B30006F0000008327850217E70100130747BFD6
:102B4000E38EE7FAE39C07FA9309450013040500B6
:102B500013850900EFD05FC897E701009387479E70
:102B60000325C40283A7070063F6A70097E70100C7
:102B700023A8A79C93054001EF50104897E7010058
:102B8000938707AC3385A70093850900EFD09FBCDE
:102B900083A704000327C40283A7C702E360F7F6F4
:102BA000EFD01F9F6FF09FF5032481018320C101A7
:102BB00083244101032901018329C100130101027A
:102BC0006F50905963020506130101FE232C81000A
:102BD000232A91002326310113040500232E11001E
:102BE00023282101EFD01FAF0327440197E70100FD
:102BF000938787B69309050093040000630AF702E0
:102C000013850900EFD09FAC8320C101032481010B
:102C10001385040003290101832441018329C10094
:102C20001301010267800000737004306F00000020
:102C30008327840217E50100130585AFE382A7FC13
:102C4000E39007FC97E701009387C78D83A70700F0
:102C50006394070697E701009387079083A707000F
:102C60008324C4021309440083A7C7021305090083
:102C7000B3B4F400EFD05FB697E701009387478CB9
:102C80000325C40283A7070093C4140063F6A700BA
:102C900097E7010023A6A78A93054001EF50D0359E
:102CA00097E701009387C799930509003385A7002B
:102CB000EFD05FAA6FF0DFF493058401EFD09FA9F6
:102CC0006FF01FF4130101FE37150000232E1100D1
:102CD000232C8100232A910023282101232631015E
:102CE000232441012322510123206101EF30C0231D
:102CF000630805229304050013050006EF30C02287
:102D00001304050063040526371600009305500AD6
:102D10002328950213850400EF3080538324040395
:102D2000B71700009387C7FFB384F400B7474C453B
:102D300093879744130A4400232AF40213050A00D8
:102D4000230C0402A3010404232604022328040400
:102D5000232A0404EFD09F9F13058401EFD01F9F07
:102D60009307A000232C040493F4C4FF23288400B9
:102D7000232CF4002322840223220404232E04049F
:102D800013060000971500009385C5EA138504001B
:102D9000EFD01F952320A4007370043017D90100D1
:102DA0001309C9798327090097D401009384C47A51
:102DB000638C070003A7040083A70400832747044C
:102DC000938717002322F70417D701001307C7774B
:102DD000832707009387170097D6010023A6F6766E
:102DE00083A704006388070A8327090097E9010085
:102DF00093890985639C070083A7040083A7C70202
:102E00006396070097D7010023A8877497D701001E
:102E10009387C77103A7070097D601009386467270
:102E20008327C40283A606001307170017D60100E4
:102E3000232EE66E2324E40463F6F60017D7010080
:102E40002320F770139527003305F500131525008F
:102E500093050A003385A900EFD0DF8F832709008F
:102E60006388070083A7040083A74704639E070CB9
:102E7000832709006384070083A70400EF2050071D
:102E800093071000630AF510631C05087370043083
:102E90006F00000097D7010023A0876C032707006D
:102EA0009307100097D9010093898979E310F7F609
:102EB000938A090017EB0100130B0B8513850A0099
:102EC000938A4A01EFD09F86E31A5BFF17E5010062
:102ED00013058583EFD09F8597EA0100938A0A84C2
:102EE00013850A00EFD09F8417E501001305458480
:102EF000EFD0DF8317E501001305C584EFD01F83F2
:102F000017E5010013054585EFD05F8297D70100D3
:102F100023A2676597D7010023AC57636FF01FEFBB
:102F20008320C1010324810183244101032901017C
:102F30008329C100032A8100832A4100032B010059
:102F4000130101026780000003A7040083A60400A8
:102F5000832747049387F7FF2322F70483A74604B8
:102F6000E39807F0736004306FF09FF00324810151
:102F70008320C101032901018329C100032A8100A3
:102F8000832A4100032B010013850400832441019F
:102F9000130101026F304011737004309307F0FF8A
:102FA00017D701002322F7580324810197D7010086
:102FB00023A6A7588320C1018324410103290101CD
:102FC0008329C100032A8100832A4100032B0100C9
:102FD00097D7010023A80756130101026FD08FC0B5
:102FE0007370043097D7010023AA07546FD0CFD154
:102FF00017D701001307075383270700938717008C
:103000002320F700678000007370043097D7010019
:103010009387C75203A707006318070217D7010059
:10302000130747520325070083A70700638C070097
:1030300097D701009387475203A707000327470448
:10304000631407026780000017D701001307C750F9
:10305000832607000327070003A74604130717006A
:1030600023A2E6046FF09FFB03A7070083A60700D7
:10307000832747049387F7FF2322F70483A7460497
:10308000E39207FC7360043067800000130101FFC6
:103090002326110023248100EFD0CFE397D701002E
:1030A0009387474A03A40700EFD04FE28320C10073
:1030B000130504000324810013010101678000004F
:1030C00097D701009387474803A507006780000052
:1030D000130101FD232611022324810223229102E0
:1030E00023202103232E3101232C4101232A5101C6
:1030F000232861012326710197D701009387874216
:1031000083A70700639A070617D7010013078743B1
:10311000832707009387170097D6010023A4F64260
:10312000832A0700638A0A0A97D701009387C73F5B
:1031300083A707009304000063FEFA0A97D90100F1
:103140009389095017DA0100130A0A4183270A00FC
:103150009306100003A7C70293172700B387E70061
:1031600093972700B389F90083A7090063F4F60257
:10317000930410006F00000297D701009387C73BAC
:1031800083A70700930400009387170017D7010057
:103190002324F73A97D701009387C73983A70700FD
:1031A00063840700930410008320C102032481027A
:1031B0001385040003290102832441028329C101EC
:1031C000032A8101832A4101032B0101832BC100C2
:1031D000130101036780000017D401001304843732
:1031E0008327040083A707006388070C73700430EB
:1031F0006F00000017D401001304C43597D90100F3
:103200009389094417DA0100130A0A3517DB010014
:10321000130B0B338327040083A707006380070881
:103220008327040083A7C70003A9C7008327490099
:10323000930B490013850B0063EAFA06EFD0CFD950
:10324000832789021305890163840700EFD0CFD853
:103250008327C90203270B0093850B0013952700D2
:103260003305F500131525003385A9006376F700B3
:1032700017D701002326F72CEFD0CFCD83270A00E4
:103280000327C90283A7C702E366F7F88327040070
:103290009304100083A70700E39407F89307F0FF57
:1032A00017D701002322F7286FF05FEA17D7010034
:1032B000232CF7266FF09FE917D701001307472942
:1032C000832704000327070097D6010023A4E628DC
:1032D00017D70100232EF72697D70100938747259C
:1032E00083A707009387170017D701002322F7242D
:1032F0008327040083A70700639A07009307F0FF62
:1033000017D701002322F7226FF01FE28327040062
:1033100083A7C70083A7C70083A7470017D701006B
:103320002324F7206FF05FE097D701009387871F72
:1033300003A7070063160700737004306F000000D6
:10334000130101FE232E1100232C8100232A91005A
:103350002328210123263101232441012322510165
:10336000232061017370043097D401009384041DFD
:1033700003A704006310071203A707001307F7FF52
:1033800097D6010023A0E61A83A70700639E070AC9
:1033900097D701009387471B83A707006386070A17
:1033A00097DA0100938ACA2917DA0100130A4A1929
:1033B00017D901001309491A930910006F00C001C1
:1033C0003385EA00EFD00FB9832709000327C40231
:1033D00083A7C7026374F70683A70A0F6380070EEB
:1033E00083A7CA0F03A4C70013058401EFD0CFBE83
:1033F000130B440013050B00EFD00FBE8327C4024C
:1034000083260A0093050B00139527003305F5006A
:1034100013152500130705003385AA00E3F2F6FA19
:1034200017D70100232EF710EFD0CFB28327090062
:103430000327C40283A7C702E360F7FA97D7010006
:1034400023AA370F6FF05FF91304000083A704006D
:10345000638C070097D701009387071083A70700A5
:1034600083A7470463980704130504008320C10160
:103470000324810183244101032901018329C1001F
:10348000032A8100832A4100032B0100130101025A
:103490006780000017D701001307070C8326070079
:1034A0000327070003A746041307170023A2E60417
:1034B0006FF09FECEF50404A6FF01FFB17D40100F4
:1034C0001304840783270400638C07028327040006
:1034D0001309100063860702EFF09FBF6306050023
:1034E00097D7010023A82705832704009387F7FFB8
:1034F00017D701002322F70483270400E39E07FC6B
:1035000097D701009387070303A7070093071000CD
:10351000E31CF7F2EFD0CF87130410006FF01FF316
:103520006304050263960500737004306F000000A9
:1035300017D70100130707FF83270700638A0700D7
:10354000737004306F000000737004306F0000006F
:10355000130101FF23248100232611008326070085
:10356000032705009386160017D60100232CD6FAF0
:1035700097D60100938606FD83A606003304B700A4
:103580002320850063F0E6046372E40263F08602A0
:1035900097D70100938747FC03A507001305450053
:1035A000EFD08FA313050400EF508032EFF0DFD788
:1035B000630E05008320C100032481001301010173
:1035C00067800000E366E4FC6FF05FFC0324810089
:1035D0008320C100130101016FC09FFB630E050032
:1035E00017D70100130707F4832707006388070034
:1035F000737004306F0000006FC09FF9130101FF6A
:1036000023261100232481000327070093070500C8
:103610001307170097D6010023A6E6F097D60100FE
:10362000938686F317D701001307C7F10327070016
:1036300003A506003304F70013054500EFD0CF992A
:1036400013050400EF50C028EFF01FCE631A0500E9
:10365000032481008320C100130101016FC05FF3C7
:103660008320C10003248100130101016780000051
:10367000130101FF232481002326110097D70100A5
:10368000938747EA83A70700130400009387170076
:1036900017D701002328F7E897D701009387C7EAD7
:1036A00083A7070063EEF51417DE0100130E0E0565
:1036B00097D20100938202F8130400001307000060
:1036C000930F10001303500A6F00C000130ECEFEBC
:1036D0006384C20F83278EFF93060700E38807FEEB
:1036E0008327CEFF83A74700232EFEFE6386C713E2
:1036F00003AFC70083A747003307E500930E000020
:10370000232EFEFE6380C70983A8C7009387480362
:10371000232017012322F70083A788042326F7011B
:103720002324F70083A7C8022328F70083A70805EE
:10373000232C0700232AF70003A808038347080067
:1037400063986704930708009387170083C60700F0
:10375000B3850741E38A66FE93D52500939505015D
:1037600093D50501231EB700938E1E001307070291
:10377000630A1F038327CEFF83A74700232EFEFE85
:10378000E394C7F983274E00232EFEFE6FF0DFF788
:1037900093050000231EB700938E1E001307070237
:1037A000E31A1FFD3304D40113175400130ECEFE89
:1037B00093060700E390C2F397D70100938787D958
:1037C00003AE070083270E006396071297D7010008
:1037D000938707D803AE070083270E00639A071C60
:1037E00017DE0100130ECEE583274E10639C0702FF
:1037F00083278E11639C072663040600232006009E
:10380000EFF09FB2130504008320C1000324810060
:10381000130101016780000083274E00232EFEFE66
:103820006FF01FED83278E1017DF0100130F0FF2CB
:1038300083A7470017D701002328F7F06386E73DE9
:1038400083A2C70083A74700B306D500930E0000EC
:1038500017D70100232AF7EE930F40001303500AF5
:103860006382E70983A8C7009387480323A0160152
:1038700023A2F60083A7880423A6F60123A4F6005A
:1038800083A7C80223A8F60083A7080523AC060077
:1038900023AAF60003A8080383470800639A673247
:1038A000930708009387170003C70700B3850741F4
:1038B000E30A67FE93D725009397070193D7070183
:1038C000239EF600938E1E0093860602638C1231AF
:1038D00083278E1083A7470017D701002326F7E61A
:1038E000E392E7F983270E1117D70100232EF7E49F
:1038F0006FF05FF783274E00130F8E0083A64700FB
:103900002322DE006380E633B307E50003A7460009
:1039100083A2C600930E00002322EE00930F200026
:103920001303500A6300EF088328C7001387480376
:1039300023A0170123A2E70003A7880423A6F70109
:1039400023A4E70003A7C80223A8E70003A70805EC
:1039500023AC070023AAE70003A8080303470800D5
:10396000631E67221307080013071700834607002A
:10397000B3050741E38A66FE13D725001317070135
:1039800013570701239EE700938E1E0093870702BB
:103990006380122383264E0003A746002322EE00F5
:1039A000E314EFF80327CE002322EE006FF0DFF7D9
:1039B00083274E00130F8E0083A747002322FE00AB
:1039C000638CE72583A2C70083A74700B306D50011
:1039D000930E00002322FE00930F20001303500AD1
:1039E0006300FF0883A8C7009387480323A016013C
:1039F00023A2F60083A7880423A6F60123A4F600D9
:103A000083A7C80223A8F60083A7080523AC0600F5
:103A100023AAF60003A808038347080063986714E5
:103A2000930708009387170003C70700B385074172
:103A3000E30A67FE93D725009397070193D7070101
:103A4000239EF600938E1E0093860602638A12134D
:103A500083274E0083A747002322FE00E314FFF8CC
:103A60008327CE002322FE006FF0DFF78327CE11DD
:103A700097DE0100938ECECE83A7470017D70100B3
:103A8000232EF7CC638AD71783AFC70083A74700DD
:103A90003307D5001303000097D6010023A0F6CC0E
:103AA000130F3000930220009308500A6388D7094F
:103AB00003A5C700930745032320A7002322F7008F
:103AC000832785042326E7012324F7008327C502E3
:103AD0002328F700832785026384070023265700E5
:103AE00083270505232C0700232AF7000328050355
:103AF00083470800639C1705930708009387170006
:103B000083C60700B3850741E38A16FF93D72500D4
:103B10009397070193D70701231EF70013031300A0
:103B200013070702638EAF028327CE1183A74700D6
:103B300097D6010023A4F6C2E39CD7F783274E1241
:103B400097D6010023ACF6C06FF09FF693070000F4
:103B5000231EF7001303130013070702E396AFFCBD
:103B600033046400E31C06C86FF09FC9930700008C
:103B7000239EF600938E1E0093860602E39A12EDB2
:103B800017DE0100130ECEAB83274E103304D40191
:103B900093165400E38E07C46FF0DFC813070000CC
:103BA000239EE700938E1E0093870702E39412DFA3
:103BB00097D701009387C79903AE07003304D40158
:103BC0009316540083270E00E38C07C06FF05FDE6E
:103BD00093070000239EF600938E1E009386060234
:103BE000E39812CF83278E113304D4019316540027
:103BF000E38407C06FF09FE783274E1217D70100B9
:103C0000232EF7B46FF05FE883270E1117D701005A
:103C1000232CF7B26FF0DFC28327CE002322FE00F1
:103C20006FF05FDA8326CE002322DE006FF0DFCD57
:103C3000130101FD2322910223202103232E3101B0
:103C4000232C4101232A51012328610123267101DC
:103C5000232611022324810297D901009389898C9C
:103C600017D901001309C99D17DA0100130A0A8D3B
:103C700097DA0100938A4A8E97DB0100938BCB8CF5
:103C800097D401009384848C130B10006F00000202
:103C900083A70900032449109387170017D7010051
:103CA0002322F788EFF04FE8631E040083A7040087
:103CB000E39007FE83270900E37AFBFEEFC05F8DE8
:103CC0006FF0DFFE7370043083270A00639E0704E1
:103CD0008327091103A4C70013054400EFC0DFAF19
:103CE00083A70B009387F7FF17D70100232EF784D4
:103CF00083A704009387F7FF17D701002328F784D1
:103D000083270A006388070083A70A0083A7470464
:103D10006398070203250403EF200039130504000C
:103D2000EF2080386FF09FF803A70A0083A70A00EE
:103D300083274704938717002322F7046FF05FF966
:103D400003A70A0083A60A00832747049387F7FF87
:103D50002322F70483A74604E39E07FA7360043026
:103D60006FF05FFB97C701009387C77B83A70700AE
:103D7000639E070E130101FF2326110023248100F7
:103D80002322910097C7010023A6077A17C70100D5
:103D90001307877C83270700B7A6A5A59386565AE5
:103DA00083A7070383A50700639ED50003A64700EA
:103DB000631AB60083A687006396C60083A7C70070
:103DC000638AD700032507008325070093854503F1
:103DD000EF30007F17C7010013078776832607009F
:103DE00017D401001304C4856F0000028327070065
:103DF00063860708832707009387F7FF97C60100AC
:103E000023A0F6748326070093972600B387D70074
:103E100093972700B307F40083A70700E38807FC04
:103E20000325070093172500B387A7009397270062
:103E30003307F4008326470093878700B307F40015
:103E400083A4460023229700638EF40283A7C40054
:103E50008320C1000324810017C70100232EF76EC1
:103E600083244100130101016780000093071000C3
:103E700017C701002320F76C6780000073700430BF
:103E80006F00000083A4440093054001EF40D0166A
:103E90003305A400232295006FF05FFB130101FEA0
:103EA00023282101232E1100232C8100232A910095
:103EB00023263101130905007370043097C40100F3
:103EC0009384C46783A7040017C401001304C46863
:103ED000639C070C6314090003290400930949003B
:103EE00013850900EFC05F8F83278902638607006F
:103EF00013058901EFC05F8E9385090017D5010076
:103F000013058585EFC01F8583A70400638807001C
:103F10008327040083A747046394070A83270400C8
:103F20006384270D83A7040063820706737004303F
:103F300083A704006398070E97C7010093878761E2
:103F400003A70700032707006310070C9307F0FF80
:103F500017C70100232AF75C83A7040063880702C0
:103F60008327040083A74704638207020327040012
:103F700083260400832747049387F7FF2322F7044F
:103F800083A7460463940700736004308320C10153
:103F90000324810183244101032901018329C100F4
:103FA0001301010267800000032704008327040037
:103FB00083274704938717002322F7046FF09FF1AC
:103FC0000327040083260400832747049387F7FF11
:103FD0002322F70483A74604E39207F473600430B6
:103FE00083270400E39027F583A704006382070674
:103FF00097C701009387075383A707006388070AC1
:10400000737004306F00000083A7070083A7C70008
:1040100083A7C70083A7470017C701002326F750CF
:104020006FF09FF3032704008327040083274704CE
:10403000938717002322F70497C7010093878751BE
:1040400003A7070003270700E30207F06FF0DFFB79
:1040500097C701009387474F17C701001307475EB3
:1040600083A70700032787116314F7028320C10188
:104070000324810197C7010023A0074E8324410137
:10408000032901018329C100130101026780000097
:10409000032481018320C1018324410103290101FB
:1040A0008329C100130101026FF0DFCB03248101DA
:1040B0008320C10183244101032901018329C10017
:1040C000130101026FC0CFCC6306050A130101FF83
:1040D0002322910097C401009384044823202101E6
:1040E0001389050083A504002326110023248100E1
:1040F00093858501EFC00FE903A504001305450072
:10410000EFC08FED9307F0FF630AF90697C7010030
:104110009387474303A4070003A7040083A707006E
:104120003304240123228700636EF40697C701003D
:104130009387474203A5070083A5040093854500A4
:10414000EFC04FE497C701009387073E83A707009E
:104150006376F40097C7010023A8873C8320C10041
:10416000032481008324410003290100130101017C
:1041700067800000737004306F00000083A50400A6
:10418000032481008320C10083244100032901000E
:1041900017C501001305455C938545001301010116
:1041A0006FC04FDB97C701009387873A03A50700CD
:1041B0000324810083A504008320C10083244100DF
:1041C0000329010093854500130101016FC08FDBB6
:1041D000630E050097C701009387C73483A70700C4
:1041E000639A0700737004306F000000737004302E
:1041F0006F000000130101FF2322910097C401000A
:104200009384843503A704009387050083A50400E5
:10421000B7060080B3E7D7002326110023248100CE
:10422000232CF7009385850113040600EFC08FD27D
:1042300003A5040013054500EFC00FDA9307F0FF54
:104240006304F40297C701009387C72F03A50700F3
:104250008320C100832441003305850003248100AD
:10426000130101016F40C06683A50400032481008F
:104270008320C1008324410017C501001305C54DEB
:1042800093854500130101016FC0CFCC6308050A77
:10429000130101FF2322910097C401009384C42BD2
:1042A000232021011389050083A504002326110082
:1042B000232481009385850113040600EFC08FC974
:1042C00003A5040013054500EFC00FD193071000AC
:1042D000630AF40697C701009387C72603A4070063
:1042E00003A7040083A707003304240123228700C7
:1042F000636EF40697C701009387C72503A50700DF
:1043000083A5040093854500EFC0CFC797C7010080
:104310009387872183A707006376F40097C701007E
:1043200023A487208320C10003248100832441002B
:10433000032901001301010167800000737004303C
:104340006F00000083A50400032481008320C100C6
:10435000832441000329010017C501001305C53F4F
:1043600093854500130101016FC0CFBE97C70100BF
:104370009387071E03A507000324810083A504007B
:104380008320C10083244100032901009385450057
:10439000130101016FC00FBF130101FF232611009C
:1043A00023248100232291008327C50003A4C70092
:1043B0006304040A9304840113850400EFC0CFC191
:1043C00097C701009387071683A70700639A07081A
:1043D0009304440013850400EFC00FC097C7010089
:1043E000938707160327C40283A7070063F6E70035
:1043F00097C7010023A6E71493172700B387E700A8
:104400009397270017C501001305852393850400A2
:104410003305F500EFC00FB497C701009387C713AA
:1044200083A707000327C4021305000083A7C70260
:1044300063FAE7009307100017C70100232CF70E5B
:10444000130510008320C100032481008324410050
:104450001301010167800000737004306F000000D9
:104460009385040017C501001305852CEFC08FAE9E
:104470006FF09FFA97C701009387C70A83A70700C9
:1044800063960700737004306F000000130101FF92
:10449000232611002324810023229100B7070080E6
:1044A0000324C500B3E7F5002320F50063080408E2
:1044B000EFC08FB29304440013850400EFC0CFB166
:1044C00097C701009387C7070327C40283A7070084
:1044D00063F6E70097C7010023A4E70693172700B8
:1044E000B387E7009397270017C50100130545150B
:1044F0003305F50093850400EFC0CFA597C70100F1
:104500009387870583A707000327C40213050000CC
:1045100083A7C70263FAE7009307100017C70100DB
:10452000232AF700130510008320C1000324810013
:10453000832441001301010167800000737004307F
:104540006F0000006304050297C70100938747FED0
:1045500003A7070097C701009387C7FE83A707003B
:104560002320E5002322F5006780000073700430EB
:104570006F0000006304050E638E050C130101FF3C
:1045800023261100232481001307050073700430D3
:1045900097C80100938888FA83A708006380070200
:1045A00097C70100938747FB83A6070083A70700EF
:1045B00083A746049387170023A2F60417C30100BC
:1045C000130343F883A70500032603009306F0FFB7
:1045D000130400006388D70417CE0100130E4EF5B4
:1045E00003250E0003280700832647006306A80062
:1045F000130410006378D6023308D6401304100069
:104600006372F80203250E00B387C7400326030038
:10461000B387D70023A0F5002320A7002322C700DB
:104620001304000083A70800638C070097C70100EC
:10463000938787F283A7070083A747046394070241
:10464000130504008320C10003248100130101012C
:1046500067800000737004306F00000073700430D6
:104660006F000000EF40402F6FF09FFD9307100098
:1046700017C701002320F7EC6780000063060500E0
:104680000325C50467800000130500006780000053
:10469000630405002326B5046780000097C7010066
:1046A000938787EB03A507006780000097C7010089
:1046B0009387C7E883A7070013051000638C0700E2
:1046C00097C70100938707E603A507001335150078
:1046D0001315150067800000630C0508130101FE27
:1046E000232A910097C40100938404E783A7040060
:1046F000232E1100232C81002328210123263101A0
:104700000327C50283A7C7026376F70483278501C1
:1047100063CC070083A7040083A6C7029307A00009
:10472000B387D740232CF50093172700B387E70002
:104730000327450117C90100130989F09397270042
:10474000B307F9006308F70283A7040083A7C70231
:104750002326F5028320C101032481018324410122
:10476000032901018329C1001301010267800000B0
:1047700067800000930945001304050013850900B4
:10478000EFC08F8583A7040017C70100130747DB1D
:104790000327070083A7C7022326F4026376F700E6
:1047A00017C70100232EF7D8139527003305F5000E
:1047B00003248101131525008320C10183244101B5
:1047C000938509003305A9008329C100032901014C
:1047D000130101026FB01FF863060502130101FF08
:1047E00023261100232481002322910097C7010072
:1047F000938787D603A40700630AA400737004306C
:104800006F00000013050000678000008327440547
:1048100063960700737004306F0000008326C402A3
:10482000032704059387F7FF232AF4046384E60033
:10483000638E0700130500008320C100032481005C
:1048400083244100130101016780000093044400A8
:1048500013850400EFB05FF80325040597C7010036
:10486000938707CE03A707009307A000B387A7404D
:104870002326A402232CF4006376A70097C7010027
:1048800023A0A7CC93054001EF30107797C7010014
:10489000938707DB3385A70093850400EFB09FEB78
:1048A000130510006FF05FF97370043097C70100B3
:1048B0009387C7C883A707006380070297C70100D3
:1048C000938787C903A7070083A7070083274704A7
:1048D000938717002322F7046780000097C7010021
:1048E0009387C7C583A70700638C070297C701009A
:1048F000938787C603A707000327470463020702BD
:1049000003A7070083A60700832747049387F7FFC1
:104910002322F70483A746046394070073600430DE
:104920006780000097C70100938707C303A60700AD
:1049300083A6070003A707009307A00083A6C6026B
:1049400003258601B387D740232CF700678000003A
:1049500097C70100938747C003A70700630A0700B2
:1049600083A6070003A746051307170023AAE6043A
:1049700003A5070067800000130101FD2320210328
:10498000232611022324810223229102232E3101A6
:10499000130905007370043097C40100938404BAAE
:1049A00083A7040017C40100130404BB639E070A15
:1049B0008327040083A78705639A070083270400E1
:1049C0001307100023AEE704639A050E83A70400C3
:1049D000638807008327040083A74704639A0714AA
:1049E0007370043083A704006394070683270400D0
:1049F00003A58705630805006302090483270400F3
:104A000023AC07048327040023AE070483A7040014
:104A1000638807008327040083A74704639207067F
:104A20008320C1020324810283244102032901025D
:104A30008329C101130101036780000003270400DB
:104A4000832787059387F7FF232CF7046FF09FFBDD
:104A50000327040083270400832747049387170054
:104A60002322F7046FF09FF8032704008327040034
:104A700083274704938717002322F7046FF05FF31F
:104A80000327040083260400832747049387F7FF46
:104A90002322F70483A74604E39407F873600430E5
:104AA0008320C102032481028324410203290102DD
:104AB0008329C1011301010367800000032504005D
:104AC0002326B10013054500EFB01FD18325C10097
:104AD0009307F0FF6380F50897C70100938787A6C7
:104AE00083A907000327040083A70700B389B9003F
:104AF0002322370163ECF90697C70100938787A546
:104B000003A507008325040093854500EFB09FC7E8
:104B100097C70100938747A183A7070063F6F900B1
:104B200097C7010023A237A1EFB09FA66FF01FEA3D
:104B30000327040083260400832747049387F7FF95
:104B40002322F70483A74604E39C07E8736004303C
:104B50006FF01FE98325040017C501001305C5BFC9
:104B600093854500EFB01FBF6FF01FFC97C7010092
:104B70009387079E03A507008325040093854500BE
:104B8000EFB05FC06FF05FFA130101FD2320210336
:104B9000232E310123261102232481022322910294
:104BA000232C41011389050093090600737004301A
:104BB00097C401009384849883A7040017C401005C
:104BC00013048499639C07140327040093072000AF
:104BD0000327C7056304F702832704001345F5FF85
:104BE00003A787053375E50023ACA70483270400DA
:104BF0001307100023AEE704639A060A83A7040094
:104C0000638807008327040083A74704639407167B
:104C10007370043083A70400639E0706638809004D
:104C20008327040083A7870523A0F9000327040036
:104C300093071000130500000327C705630EF70054
:104C4000832704001349F9FF1305100003A7870504
:104C50003379E90023AC27058327040023AE07043A
:104C600083A70400638807008327040083A7470401
:104C70006392070C8320C102032481028324410232
:104C8000032901028329C101032A810113010103C0
:104C9000678000000327040083270400832747045C
:104CA000938717002322F7046FF05FF703250400B2
:104CB0002326D10013054500EFB01FB28326C100A3
:104CC0009307F0FF638AF60C97C7010093878787E5
:104CD00003AA07000327040083A70700330ADA00AA
:104CE000232247016368FA0C97C7010093878786E0
:104CF00003A507008325040093854500EFB09FA816
:104D000097C701009387478283A707006370FA0A59
:104D100097C7010023AA47816F00400903270400B9
:104D20008327040083274704938717002322F7046F
:104D30006FF09FE9032704008326040083274704BC
:104D40009387F7FF2322F70483A74604E39407F22F
:104D5000736004308320C102032481028324410252
:104D6000032901028329C101032A810113010103DF
:104D7000678000000327040083260400832747047C
:104D80009387F7FF2322F70483A74604E39207E8FB
:104D9000736004306FF0DFE78325040017C501005E
:104DA0001305859B93854500EFB0DF9AEFB04FFE6A
:104DB0006FF0DFE497B701009387877903A50700B9
:104DC0008325040093854500EFB0DF9B6FF01FFE45
:104DD000630A050C130101FF23261100232481001F
:104DE00023229100232021017370043097B4010025
:104DF0009384C47483A7040063960708638606003F
:104E00008327850523A0F60093070600930620005C
:104E10000326C505232ED5041387050013040500BA
:104E20006382D70A63F4F608930530006388B700FD
:104E3000930540006396B700630CD610232CE4045E
:104E400093071000630CF6081304100083A70400F6
:104E5000638C070097B701009387077083A707004B
:104E600083A7470463980706130504008320C10045
:104E7000032481008324410003290100130101015F
:104E80006780000097B701009387076D03A70700AD
:104E900083A7070083274704938717002322F7047B
:104EA0006FF0DFF5737004306F00000093061000A0
:104EB000E398D7F88327850533E7B700232CE5046B
:104EC0006FF01FF88327850593871700232CF504BF
:104ED0006FF01FF7EF3050286FF01FF913094400EF
:104EE00013050900EFB05F8F97B7010093874765FF
:104EF0000325C40283A7070063F6A70097B7010044
:104F000023A0A76493054001EF30100F97B701006D
:104F1000938707733385A70093050900EFB09F833C
:104F20008327840263860700737004306F000000DB
:104F300097B701009387476283A707000327C4023E
:104F400083A7C702E3F2E7F0EFB08FE46FF0DFEF83
:104F5000130400006FF09FEF63080508130101FEC2
:104F6000232C8100232A91002328210123263101AB
:104F70002324410123225101232E1100930907000C
:104F8000138A060093040600138905001304050024
:104F9000EFB04FF4930A050063060A0083278405E7
:104FA0002320FA000327C40593072000232EF404CE
:104FB0006380F40463FA9710930630006388D4008A
:104FC000930640006396D400630CF70E232C24054F
:104FD000930710006312F70A832784026382070293
:104FE000737004306F000000737004306F000000B5
:104FF0008327840593871700232CF4046FF05FFD4B
:1050000097B701009387075283A707006390070AA9
:105010009304440013850400EFB00FFC97B7010020
:10502000938707520325C40283A7070063F6A700EE
:1050300097B7010023A6A75093054001EF30C07B2E
:1050400097B701009387C75F938504003385A70056
:10505000EFB04FF097B701009387075083A7070081
:105060000327C40283A7C70263F8E7006386090029
:105070009307100023A0F9001304100013850A0001
:10508000EFB0CFE4130504008320C10103248101A4
:1050900083244101032901018329C100032A8100DE
:1050A000832A4100130101026780000093058401F7
:1050B00017B501001305C567EFB0CFE96FF09FF991
:1050C000130400006FF09FFB93071000E392F4F0CD
:1050D0008327840533E92701232C24056FF05FEF34
:1050E000630A050E130101FE232C8100232A91007F
:1050F0001304050023263101232E1100232821014A
:1051000093840500EFB00FDD930720008326C405CC
:10511000232EF40483278405130710009309050048
:1051200093871700232CF4046396E60883278402F0
:1051300063860700737004306F00000097B70100AA
:105140009387473E83A70700639A07081309440023
:1051500013050900EFB04FE897B701009387473E6A
:105160000325C40283A7070063F6A70097B70100D1
:1051700023A8A73C93054001EF30006897B70100D2
:105180009387074C930509003385A700EFB08FDCA8
:1051900097B701009387473C83A707000327C40202
:1051A00083A7C70263F8E700638604009307100033
:1051B00023A0F400032481018320C1018324410141
:1051C00003290101138509008329C100130101028C
:1051D0006FB0CFCF737004306F000000930584016F
:1051E00017B501001305C554EFB0CFD66FF05FFAC5
:1051F00093070500630805067370043017B70100B4
:105200001307C73383260700639E060203A6C7055C
:1052100093062000130500006316D60023AE070492
:105220001305100083270700638C070097B7010060
:105230009387873203A7070003274704631C0702ED
:105240006780000097B601009386063103A606002A
:1052500083A6060083264604938616002322D604DE
:105260006FF0DFFA97B701009387072F83A7070036
:105270006FF09FF803A7070083A607008327470462
:105280009387F7FF2322F70483A74604E39A07FADC
:105290007360043067800000130101FB2322910436
:1052A00023202105232C4103232A510323286103B2
:1052B000232671032326110423248104232E310382
:1052C00023248103232291032320A10317B9010082
:1052D0001309892917BB0100130B4B2897B4010050
:1052E0009384042897BA0100938ACA27130A1000EE
:1052F000930B90008327090003A707006306071696
:1053000083A7C70083A90700EFD09FCEEFD0DFCFE0
:1053100083270B00130C05006368F50C97B7010099
:1053200023AEA722130600006376352303A50400ED
:10533000B3858941EFC09F9EEFD01FFF630605161E
:1053400003A50400930600001306000093058100E6
:10535000EFC08FADE30005FA83278100E3C207FEAB
:105360008329010183A7490163860700138549004A
:10537000EFB08FC6EFD05FC983270B00130C050079
:105380006362F50C8327810017B701002328871D6E
:10539000E3E8FBFAB317FA0013F7072163100720BD
:1053A00013F7770C6316072A93F70702E38A07F8C7
:1053B00013850900EF00504F6FF09FF883A7C700D7
:1053C00003A4C70083AC07009309440013850900B8
:1053D000EFB08FC08327440213050400E780070065
:1053E0008327C4016386470D8327090003A70700AD
:1053F000E31607FC03A70A0097B6010023A086174F
:1054000097B6010023A0F61697B7010023AEE71464
:10541000EFD09FF16FF0DFF283A7C70003A4C700AE
:1054200003AD0700930C440013850C00EFB0CFBA16
:105430008327440213050400E78007008327C40183
:10544000638C470B8327090003A70700E31607FCBB
:1054500003A70A0097B6010023A6F61097B701002C
:1054600023A4E7106FF01FF2EFD09FB8EFD0DFB9A1
:1054700083270B00130C0500E368F5F683A70A00E9
:1054800003A504009309000003A60700B385894122
:1054900017B701002324870D13361600EFC01F88AD
:1054A000EFD09FE8E31E05E8EFB08F8E6FF05FE965
:1054B0008327840193850900B387FC0063E2FC081D
:1054C00083A7040063860702232A0100232C91018D
:1054D000232E8100EFF08F9D03A5040093060000AA
:1054E0001306000093054101EFB0DFACE31E05EEAB
:1054F000737004306F0000008327840193850C00D3
:10550000B307FD006362FD0883A7040063860702FA
:10551000232A0100232CA101232E8100EFF00F99F3
:1055200003A5040093060000130600009305410143
:10553000EFB05FA8E31805F0737004306F0000004F
:10554000032509002322F40023288400EFB08FA351
:105550006FF09FE9EFD05FDD8327090083A7C700C5
:1055600003A4C700930C440013850C00EFB0CFA632
:105570008327C401638A4705832744021305040077
:10558000E78007006FF0DFDB032509002322F4002A
:1055900023288400EFB00F9F6FF0DFEA8327C1005C
:1055A00023ACF9006382070AB387870123A2F900BD
:1055B00023A83901938549006362FC0803A50A000A
:1055C000EFB04F9C6FF0DFD783278401232884003E
:1055D0003387F9002322E400636AEC04330C3C4176
:1055E000636EFC0283A7040063860702232A01007E
:1055F000232C3101232E8100EFF04F8B03A50400F3
:10560000930600001306000093054101EFB09F9A36
:10561000E31405F6737004306F00000003A50A0060
:1056200093850C00EFB00F966FF01FF5032509006E
:1056300093850C00EFB00F956FF01FF40325090060
:10564000EFB04F946FF0DFCF737004306F00000045
:105650008327C10083A6890123A839013387D70096
:1056600023A2E9006362EC06B307FC4063EAD706B5
:1056700083A7490213850900E780070083A7C901B2
:10568000E39047CD83A689018327C10003A70400C7
:10569000B387D70063060702232A0100232CF100F9
:1056A000232E3101EFF08F8003A504009306000044
:1056B0001306000093054101EFB0DF8FE31205C828
:1056C000737004306F0000006374FC00E372F7FA3B
:1056D0000325090093854900EFB0CF8A6FF05FC6BC
:1056E00003A50A0093854900EFB0CF896FF05FC52D
:1056F000130101FF2324810023261100232291009E
:105700002320210117B40100130484E5EFF0CF99A1
:105710008327040063840704EFF04F9C8327040071
:10572000638A070293080000130800009307000033
:1057300013072000930600001306004097B50100F0
:105740009385C5C717050000130545B5EFC01F9E1B
:1057500063140506737004306F00000017B9010070
:105760001309C90013050900EFA05FFC97B40100FD
:105770009384040113850400EFA05FFB130600006F
:105780009305C0001305400097B7010023AE27DD45
:1057900097B7010023A897DCEFB08FC817B70100B7
:1057A0002320A7DC6306050297B50100938585C019
:1057B000EFC08FC36FF05FF68320C1000324810028
:1057C00083244100032901001301010167800000C7
:1057D000737004306F000000638A050A130101FD35
:1057E000232A5101930A05001305C00223248102D4
:1057F0002322910223202103232E3101232C410156
:1058000023261102232861012326710113090700B1
:1058100093890600130A060093840500EF00C07008
:1058200013040500630C0502EFF00F8897B7010021
:10583000938707D383A70700638E0704EFF00F8ACF
:105840001305440023205401232C9400232E4401EB
:105850002320340323222403EFA05FEF1305040069
:105860008320C1020324810283244102032901020F
:105870008329C101032A8101832A4101032B0101EC
:10588000832BC10013010103678000007370043093
:105890006F00000097BB0100938B4BED13850B004D
:1058A000EFA0DFE817BB0100130B8BED13050B0016
:1058B000EFA0DFE7130600009305C00013054000CA
:1058C00097B7010023A277CB97B7010023AC67C934
:1058D000EFB00FB517B701002324A7C8630A05006E
:1058E00097B50100938505ADEFC00FB06FF01FF5C0
:1058F000737004306F000000630E0506130101FE93
:10590000232C8100232E1100232A910017B40100BB
:10591000130404C5832804001308050013050000C0
:1059200063800804930407002322B1001387060054
:105930002324C100232601019306500063C0B6044E
:10594000EFE0DFD693072000630EF5040325040083
:10595000930600001306000093054100EFB08FE5A9
:105960008320C10103248101832441011301010229
:1059700067800000737004306F00000093054100E1
:10598000930600001306070013850800EFB05F9828
:105990008320C101032481018324410113010102F9
:1059A00067800000032504009306000013860400AE
:1059B00093054100EFB00FE06FF09FFA630605001A
:1059C0000325050067800000737004306F0000003D
:1059D00063160500737004306F000000130101FFAF
:1059E000232611002324810013040500EFE0DFEBE0
:1059F000032544013334A000EFE05FEE13050400FB
:105A00008320C1000324810013010101678000008D
:105A100063160500737004306F000000130101FF6E
:105A2000232481001304050023261100EFE0DFE7A3
:105A300003240402EFE09FEA8320C1001305040061
:105A40000324810013010101678000006316050033
:105A5000737004306F000000130101FF23248100E4
:105A600023229100138405009304050023261100CE
:105A7000EFE09FE323A08402032481008320C10080
:105A800083244100130101016FE05FE5130101FF71
:105A90001305C0012324810023261100EF00C04814
:105AA00013040500630805002320050013054500C5
:105AB000EFA0DFC7130504008320C1000324810089
:105AC000130101016780000063020502B70700FFB0
:105AD000B3F7F50063860700737004306F000000B1
:105AE000639A0500737004306F0000007370043017
:105AF0006F000000130101FE232C810023282101E7
:105B0000232631012324410123225101232E110098
:105B1000232A91009309070013890600930A0600BF
:105B200013840500130A0500EFE05FB86318050051
:105B300063860900737004306F000000EFD04FCB14
:105B400083240A00B3779400631209046382070474
:105B500063880A009347F4FFB3F797002320FA0005
:105B6000EFD08FFC8320C101032481011385040041
:105B700003290101832441018329C100032A8100F3
:105B8000832A41001301010267800000E302F4FC54
:105B9000E38809FCB335500193958501630609003C
:105BA000B7070004B3E5F50013860900B3E58500E7
:105BB00013054A00EFE0CFE1EFD00FF763140500C3
:105BC000EFA01F9DEFE01FD6931765009309050016
:105BD00063DA0700B70400019384F4FFB3F499007B
:105BE0006FF05FF8EFE05FCC83290A00B3773401F0
:105BF00063100902638A070063880A009347F4FF71
:105C0000B3F737012320FA00EFE05FCD6FF09FFC80
:105C1000E31CF4FE6FF05FFE630C0500B70700FFA6
:105C2000B3F7F500638A0700737004306F0000005B
:105C3000737004306F000000130101FF2324810002
:105C400013040500232611002322910023202101A3
:105C500013890500EFE05FC5832404009345F9FF35
:105C6000B3F795002320F400EFE05FC78320C10065
:105C700003248100138504000329010083244100CB
:105C80001301010167800000130101FF232481003B
:105C90001304050023261100EFA0DFA30324040052
:105CA000EFA0DFA28320C1001305040003248100BC
:105CB0001301010167800000630C0500370700FF36
:105CC000B3F7E500638A0700737004306F000000CB
:105CD000737004306F0000006F20D04AB70700FFD8
:105CE000B377F60063860700737004306F0000001E
:105CF00063160600737004306F000000130101FE8C
:105D0000232C810023282101232631012324410152
:105D1000232E1100232A9100138906009389050080
:105D2000130A050013040600EFE05F98631E0504E4
:105D300063060900737004306F000000EFD04FABB2
:105D400083240A009385090013050A00B3E499002F
:105D5000EFF09FF6B3779400630AF40883240A00F7
:105D6000EFD08FDC8320C10103248101138504005F
:105D700003290101832441018329C100032A8100F1
:105D80001301010267800000EFD08FA683240A0070
:105D90009385090013050A00B3E43401EFF0DFF145
:105DA000B3F7840063848704E30A09FAB7050005A2
:105DB00013060900B365B40013054A00EFE04FC1B4
:105DC000EFD08FD663140500EFA08FFCEFE09FB5F6
:105DD000931765009304050063D40702B707000119
:105DE0009387F7FFB3F4F4006FF0DFF783270A001F
:105DF0001344F4FFB3F787002320FA006FF05FF637
:105E0000EFE09FAA83240A00B37794006398870089
:105E10009347F4FFB3F797002320FA00EFE01FAC9D
:105E20006FF0DFFB130101FF232481002326110003
:105E30001304050023229100EFD08F9B8327440099
:105E400063860702032504019304C40063189500C8
:105E50006F0080030325040163089502B705000263
:105E6000EFE04FE183274400E39607FE13050400AB
:105E7000EF008023032481008320C100832441009C
:105E8000130101016FD04FCA737004306F0000001E
:105E9000630C0500370700FFB3F7E500638A0700CE
:105EA000737004306F000000737004306F000000E6
:105EB0006F20502D630C0500B70700FFB3F7F50006
:105EC000638A0700737004306F0000007370043041
:105ED0006F000000130101FF2324810023229100A1
:105EE000232611001304050093840500EFE0DF9BD7
:105EF0000327040093C7F4FFB377F7002320F400CF
:105F0000032481008320C100832441001301010187
:105F10006FE0DF9C630605000325850167800000B4
:105F20001305000067800000130101FF2324810096
:105F30002326110013040500EFD08F8B97A70100D3
:105F40009387C76283A70700639C0704B797010084
:105F500017B70100130747849387C7FF97A601006F
:105F600023ACE66017A701002326F76017B70100EE
:105F70002326F78297A701009387875F17B7010051
:105F8000232CF7809307100017A701002328075E32
:105F900017A70100232E075C17A701002328F75C31
:105FA00063120402EFD04FB8EF10C060130400007A
:105FB000130504008320C1000324810013010101A3
:105FC0006780000013058400937735006398070C01
:105FD000B79701001307F5FF9387A7FFE3E4E7FCFA
:105FE00097A601009386465983A706006F004001DB
:105FF00003A70700630A07009386070093070700BB
:1060000003A74700E366A7FE17A70100130747563B
:10601000E38AE7F803A7070013060001138487004B
:1060200023A0E60003A74700B306A740637ED6027D
:106030003388A7002322D80023A2A7008325480085
:1060400097A60100938646536F00800093060700D1
:1060500003A7060003264700E36AB6FE2320E800F4
:1060600023A0060103A7470097A701009387875342
:1060700083A70700B387E74017A701002324F7523F
:10608000EFD08FAAE30204F2130504008320C100BD
:106090000324810013010101678000001375C5FF0F
:1060A000130545006FF0DFF263080506130101FFD9
:1060B000232481002326110013040500EFC05FF3A1
:1060C000930584FF0326C4FF17A701001307C74ADF
:1060D0006F008000138707008327070083A647000F
:1060E000E3EAC6FE232CF4FE2320B70097A70100A5
:1060F0009387474B03A707008327C4FF032481002E
:106100008320C100B387E70017A70100232CF748BD
:10611000130101016FD04FA16780000097A7010014
:106120009387474803A50700678000006780000049
:106130003367B50013773700930705006312070430
:106140009308D6FFB30815011307050093860500D1
:106150006378150303A806001307470093864600DB
:10616000232E07FFE36817FF9347F5FFB387170157
:1061700093F7C7FF93874700B385F500B307F50092
:106180003306C50063F4C70C9386450013884700A7
:10619000B3B6D70033B8050133E7F50093C6160050
:1061A0001348180013773700B3E6060113371700BA
:1061B0003377D700330EF64093861700630807063F
:1061C0001337AE006314070613532E00138805001F
:1061D00093860700130700008328080013071700A1
:1061E0001308480023A0160193864600E36667FE65
:1061F0001377CEFFB385E500B387E7006306EE04AF
:1062000083C60500138717002380D700637EC7026B
:1062100083C6150013872700A380D7006376C702C3
:1062200003C725002381E70067800000B307F6401D
:10623000B387F5009385150003C7F5FF9386160015
:10624000238FE6FEE398F5FE67800000678000007C
:10625000B367C50093F73700B308C5006382070E24
:1062600063761511B307A04093F737001387370003
:106270009306500093F5F50F130815003383A840DB
:106280001306F6FF6374D700130750006368E60E29
:106290006380070E2300B50013071000638EE7002C
:1062A000A300B50013073000130825006396E7002C
:1062B000130835002301B5001396850033E6C500A9
:1062C000139705013367E6003303F3409396850186
:1062D000B366D70013562300B307F5001307000079
:1062E00023A0D7001307170093874700E36AC7FE70
:1062F0001377C3FFB307E8006300E3082380B70008
:1063000013871700637C1703A380B7001387270048
:10631000637617032381B700138737006370170371
:10632000A381B70013874700637A17012382B70060
:106330001387570063741701A382B70067800000BA
:1063400093F5F50F13978500B365B7001397050113
:106350003367B700E37415FF930705009387470081
:1063600023AEE7FEE3EC17FF6780000067800000C4
:10637000130805006FF05FF46780000093070500C5
:106380006FF0DFF78347050013070500638C0700F4
:106390001305150083470500E39C07FE3305E54020
:1063A00067800000130500006780000013051500DA
:1063B0008347F5FF9385150003C7F5FF6388070042
:1063C000E386E7FE3385E74067800000930700001F
:1063D0006FF05FFF930705009385150003C7F5FF76
:1063E00093871700A38FE7FEE31807FE678000007E
:1063F00083460500930700026398F6001305150015
:1064000083460500E38CF6FE938756FD93F7D70F7E
:106410006380070493070500930500006388060462
:106420001305000093871700138606FD1317250038
:1064300083C607003305A700131515003305A60012
:10644000E39206FE638405003305A04067800000E8
:10645000938536FD8346150093B515009307150007
:10646000E39006FC130500006FF0DFFD130500004C
:106470006780000083A705002380A70083A705008D
:106480009387170023A0F5006780000097A60100FE
:106490009386060F83A7060017370300130787327A
:1064A00013861700B307F7002380A70097A5010004
:1064B00023A8C50C9307A000630AF5009307000406
:1064C0006308F6001305000067800000E30C06FE79
:1064D000370610F0130717008347F7FF2320F6F065
:1064E00083A706009387F7FF97A5010023AAF50865
:1064F000E39207FE1305000067800000130101EB23
:106500002322911423202115232A5113232481139C
:106510002326111423248114232E3113232C4113F9
:106520002328611323267113232291132320A113FF
:10653000232EB11193040500138905002326C10001
:10654000130C5002930A9000834709006388870365
:10655000638C070603A404006F00800063860706AF
:106560002300F40003A40400130919001304140009
:1065700023A0840083470900E39287FF03461900A4
:106580009308190093860800130D00029309F0FF89
:10659000130AF0FF13080000130550059307D6FDFA
:1065A00093F7F70F13891600636EF53A17A70100EA
:1065B000130747A593972700B387E70083A7070032
:1065C000B387E700678007008320C1140324811488
:1065D00083244114032901148329C113032A81133D
:1065E000832A4113032B0113832BC112032C811225
:1065F000832C4112032D0112832DC11113010115AA
:1066000067800000930C8000232401009307100092
:1066100063DA071D8327C10003A40400938B77006E
:1066200093F68BFF03AB060083A946009387860091
:106630002326F10013860C009306000013050B00BF
:1066400093850900EF10504B2328A1009307000009
:1066500063803733930D4101930B100013860C00B8
:106660009306000013050B0093850900EF10006BE3
:106670009306000013860C00130B05009389050098
:10668000EF1090478327810023A0AD0093861B0065
:10669000938D4D0063863701938B06006FF01FFCCE
:1066A000E37C9BFF63D24603930704002380A7018A
:1066B00003A40400130AFAFF9307140023A0F400B4
:1066C00013840700E3C446FF93962B009307010150
:1066D000B386D7006F008002938777052300F4000C
:1066E00003A40400938BFBFF93871B001304140087
:1066F00023A084009386C6FFE358F0E483A7060036
:10670000E3ECFAFC938707036FF05FFD83A70400B7
:10671000930600030327C1002380D70083A704004A
:1067200093064700930C00011386170023A0C400B2
:1067300013068007A380C70003A4040023240100DC
:10674000930707001304140023A0840003AB070081
:10675000930900002326D1006FF0DFED8327C100ED
:1067600083AC0700938B470063880C28635C40254B
:106770009307D002631EFD2083C70C0063880702C5
:1067800063D8092483A60400938C1C00130AFAFF23
:106790002380F60003A404001304140023A0840043
:1067A00083C70C00E39E07FC6352400303A404006C
:1067B000930700022300F40003A40400130AFAFF65
:1067C0001304140023A08400E3160AFE232671019B
:1067D0006FF09FD72324010093071000930CA000B3
:1067E000E3CA07E38327C10003A40400938647009C
:1067F0006FF0DFF503C61600930609006FF01FDA8D
:1068000083A70400930650022380D70003A404004A
:106810001304140023A084006FF01FD3930C000115
:10682000232401006FF09FDE8327C10003C61600FA
:106830009306090083A90700938747002326F100E8
:10684000E35E0AD4138A09009309F0FF6FF01FD5A5
:1068500003C61600130DD002930609006FF01FD473
:106860009347FAFF93D7F74103C61600337AFA002D
:10687000930609006FF09FD203C61600130D0003A4
:10688000930609006FF09FD183C51600930906FD9A
:1068900093060900938705FD13860500E3E2FAFAE3
:1068A00093972900B38937019386160093991900AD
:1068B000B389B90083C50600938909FD938705FD57
:1068C00013860500E3FEFAFC6FF09FF70327C10073
:1068D00083A7040083260700130747002326E1004F
:1068E0002380D70003A404001304140023A0840011
:1068F0006FF09FC59307100063D4070F8327C10073
:106900009386770093F686FF938786002326F1000F
:1069100083A9460083A7060063DE090E83A6040050
:106920001306D002B307F0402380C60003A404007E
:10693000B336F000B30930411304140023A08400DF
:10694000138B0700B389D940930CA00023240100C6
:106950006FF05FCE03C616001308180093060900F7
:106960006FF0DFC383A70400138908006FF09FE96D
:10697000E3729BCF93071000930B00009306100067
:10698000E3C447D36FF05FD497AC0100938C8CA322
:106990009385090013850C00EF009060330AAA402C
:1069A0006352400303A404002300A40103A40400D1
:1069B000130AFAFF1304140023A08400E3160AFE4E
:1069C000130A000083C70C00E38207E0E3CC09DA76
:1069D0009389F9FF1307F0FFE396E9DA6FF0DFDC44
:1069E0008327C1009386470083A707002326D10091
:1069F00093D9F7416FF05FF2635640019307D002DD
:106A0000E314FDF897AC0100938CCC9B93078002B4
:106A10006FF01FD7138B0700930CA00023240100F5
:106A200003A404006FF01FC1130101EB232E3113E7
:106A3000B70900409387F9FF23248114232291147E
:106A4000232C4113232A511323261114232021150B
:106A500023286113232671132324811323229113E6
:106A60002320A113232EB111130A05002324B10002
:106A700017A401001304C4B0973A0300938A8AD480
:106A8000979401009384846D2326F10093055002AE
:106A90001305A00013080004B70610F083470A008E
:106AA000638EB7046388070A03270400130A1A00D9
:106AB000130617003387EA0097A8010023A2C8AC89
:106AC0002300F7006380A708E31A06FD17370300C9
:106AD000130747CF130717008347F7FF23A0F6F0EC
:106AE000832704009387F7FF17A60100232AF6A83F
:106AF000E39207FE83470A00E396B7FA83461A003B
:106B000013051A0013070500930B0002130BF0FF87
:106B1000130CF0FF13080000930550059308900034
:106B20009387D6FD93F7F70F130A170063ECF5442C
:106B300093972700B387970083A70700B387970031
:106B400067800700173703001307C7C7E31406F869
:106B50006FF0DFF48320C1140324811483244114D3
:106B6000032901148329C113032A8113832A4113A2
:106B7000032B0113832BC112032C8112832C41128E
:106B8000032D0112832DC11113010115678000002F
:106B9000930C8000130D00009307100063DA0721A7
:106BA000832781009387770093F787FF83AD0700E2
:106BB00003AB4700138787002324E10013860C00F2
:106BC0009306000013850D0093050B00EF10C072B3
:106BD0002328A10063086D451309410193091000A2
:106BE00013860C009306000013850D0093050B001F
:106BF000EF10C01213860C0093060000930D0500E1
:106C0000138B0500EF10406F2320A9009389190012
:106C100013094900E3166DFDE3F49DFD130600041E
:106C2000B70610F063D48903832704001387170085
:106C3000B387FA0097A5010023A4E5942380770188
:106C4000630AC706130CFCFFE3C089FF8327C1005A
:106C50001305C10093089000B386F90093962600AF
:106C600093070101B386D7001308A00013030004A3
:106C7000370610F0E38CA6E083A706009305000317
:106C800063F4F8009305700503270400B387B70089
:106C9000930517003387EA0017AE01002322BE8E4A
:106CA0002300F70063860737638C65329386C6FF3F
:106CB0006FF05FFC173703001307C7B01307170007
:106CC0008347F7FF23A0F6F0832704009387F7FF9D
:106CD00097A5010023A6F58AE39207FE130CFCFF9B
:106CE0006FF09FF683270400130600041387170034
:106CF00097A5010023A6E588B386FA009305000353
:106D00002380B6006308C7509387270097A6010029
:106D100023A8F6863387EA00930680072300D7006E
:106D200017370300130707AAB70610F06392C702CC
:106D3000130717008347F7FF23A0F6F0832704000B
:106D40009387F7FF17A60100232CF682E39207FE34
:106D500083278100930C0001130D000093874700E7
:106D600003278100130B0000832D07002324F1006B
:106D70006FF0DFE48327810083AC070013894700AD
:106D8000638E0C4C6358802B9307D0026394FB3EB8
:106D900003C70C00930507006314072A6F00002F38
:106DA00093071000930CA000130D0000E3CA07DF47
:106DB00083278100938747006FF09FFA8327810024
:106DC0008346170013070A0003AB070093874700A9
:106DD0002324F100E3560CD4130C0B00130BF0FF2B
:106DE0006FF01FD483461700930BD00213070A00DD
:106DF0006FF01FD39347FCFF93D7F74183461700EB
:106E0000337CFC0013070A006FF09FD18346170004
:106E1000930B000313070A006FF09FD0034617007F
:106E2000138B06FD13070A00930706FD9306060061
:106E3000E3E2F8FA93172B00B387670113071700F3
:106E400093971700B387C70003460700138B07FD0E
:106E5000930706FD93060600E3FEF8FC6FF09FF72C
:106E600083258100832704001306A00003A70500E3
:106E700093861700B387FA00179501002322D57077
:106E80002380E700138945006300C7369307000499
:106E90006384F62A232421016FF05FBF930710005B
:106EA00063DE07358327810013877700137787FF19
:106EB000930787002324F100032B47008327070053
:106EC00063560B3E032704001306000493061700C5
:106ED0009795010023A6D56A3387EA009305D0026F
:106EE0002300B700638CC638B307F0403337F00097
:106EF000330B6041938D0700330BEB40930CA000E4
:106F0000130D00006FF09FCB834617001308180085
:106F100013070A006FF0DFC08346170013070A004B
:106F20006FF01FC083270400930600041387170027
:106F3000179601002326E664B387FA001306500271
:106F40002380C700E314D7B41737030013078787DC
:106F5000B70610F0130717008347F7FF23A0F6F0DA
:106F6000832704009387F7FF17960100232AF66012
:106F7000E39207FE6FF09FB1930C0001130D000028
:106F80006FF09FC18327040093060004130A0500D5
:106F900013871700179601002324E65EB387FA00D3
:106FA000130650022380C700E312D7AE1737030041
:106FB00013074781B70610F0130717008347F7FF41
:106FC00023A0F6F0832704009387F7FF17960100AC
:106FD0002328F65AE39207FE130A05006FF01FAB51
:106FE000172703001307077E130717008347F7FFD0
:106FF0002320F6F0832704009387F7FF979501007D
:1070000023A0F558E39207FE9386C6FF6FF09FC654
:10701000172703001307077BE39805FC9386C6FF39
:107020006FF05FC5E3FA9DBB930910006FF01FBFBF
:10703000130C000003C70C0093050700E30C07E4E2
:107040009308F0FF1305A00013080004B70610F022
:10705000635E0B0C8327040013861700B387FA00C6
:1070600017930100232EC3502380E7006382A508F5
:107070006308060B938C1C0003C70C00130CFCFF69
:1070800093050700E31607FCE35680E1832704001D
:107090009305000213060004B70610F06F00C0004D
:1070A000130CFCFFE3080CDE13871700B387FA000C
:1070B0002380B700179501002324E54C93070700B0
:1070C000E310C7FE172703001307C76F1307170046
:1070D0008347F7FF23A0F6F0832704009387F7FF89
:1070E00017950100232EF548E39207FE6FF05FFB32
:1070F000172703001307076DE30E06F613071700A3
:107100008347F7FF23A0F6F0832704009387F7FF58
:10711000179601002326F646E39207FE6FF09FF5CF
:10712000172703001307076A6FF05FFD130BFBFFC0
:10713000E3121BF36FF05FF517270300130787684F
:10714000B70610F0130717008347F7FF23A0F6F0E8
:10715000832704009387F7FF179601002322F64246
:10716000E39207FE232421016FF05F92979C0100B8
:10717000938C4C2593050B0013850C00EF004062A7
:10718000330CAC40E35880EB832704001306000463
:10719000B70610F06F00C000130CFCFFE30A0CE808
:1071A00013871700B387FA002380770197950100B2
:1071B00023A8E53C93070700E310C7FE1727030049
:1071C00013074760130717008347F7FF23A0F6F064
:1071D000832704009387F7FF9795010023A2F53AD0
:1071E000E39207FE6FF05FFB172703001307875D2D
:1071F000E39806F4232421016FF05F89832781003F
:107200001387470083A707002324E10013DBF7411E
:107210006FF01FCB172703001307C75AB70610F0EC
:10722000130717008347F7FF23A0F6F08327040016
:107230009387F7FF179601002324F634E39207FEA5
:107240009307100017970100232CF732930780074C
:10725000172703002308F7566FF09FAF635680018E
:107260009307D002E394FBF0979C0100938C8C155C
:1072700013078002930580026FF09FDC97260300BE
:1072800093864654370610F09386160003C7F6FF20
:107290002320E6F0032704001307F7FF979501006A
:1072A00023A0E52EE31207FE6FF01FC4938D0700A5
:1072B000930CA000130D00006FF05F90B70710F063
:1072C00023A0A7F26F000000130101FC1303410289
:1072D0002322B10293050300232E11002324C102AF
:1072E0002326D1022328E102232AF102232C0103C1
:1072F000232E110323266100EFF00FF38320C10139
:10730000130500001301010467800000130101FB55
:1073100013038103232481022326A100232CC1020D
:1073200013040500130603001305C10023261102F0
:107330002322F104232ED1022320E104232401057A
:1073400023261105232E6100EFF04F9B8327C100F8
:10735000238007000325C1008320C1023305854037
:10736000032481021301010567800000B70710F0B4
:1073700083A647F403A607F403A747F4E31AD7FE4E
:10738000B7160000938606FAB306D60033B6C600D9
:10739000B305E60023A4D7F423A6B7F46780000062
:1073A000B70710F003A747F403A607F483A647F432
:1073B000E31AD7FEB7160000938606FAB306D60086
:1073C00033B6C60023A4D7F4B305E60023A6B7F46A
:1073D0009307000873A0473067800000130101FF86
:1073E00023248100232611001304A0001304F4FFBA
:1073F000EF00402FE31C04FE8320C1000324810022
:107400001301010167800000130101FF23248100A3
:1074100023261100979701009387071717940100FF
:107420001304441603A70700832704001306F07C07
:1074300093064706938747069795010023A6D51420
:107440009795010023A0F514634AD6008320C1005C
:10745000032481001301010167800000130747899D
:107460009797010023A2E712EF00C02F93071000A7
:107470006316F50203270400B71700009387F77619
:1074800013050000E3D4E7FCEFF05FE30324810081
:107490008320C100130101016FB09FB41795010053
:1074A0001305C5F2EFF05FE213052000EFF01FE1D6
:1074B000032481008320C100130101016FB05FB27A
:1074C00017950100130505F26FF01FE017950100F5
:1074D0001305C5F16FF05FDF130101FF2324810065
:1074E0002322910023261100B714000017940100F5
:1074F000130444F093878438130000009387F7FF48
:10750000E39C07FE13050400EFF01FDC6FF09FFE05
:10751000130101FF2326110023248100EF008014B2
:10752000170700001307C7EB9306000013061000AF
:107530009305200317950100130545ECEFE0CFA953
:1075400013040500EFB05FAC13060500130504003B
:10755000032481008320C10013070000930600006C
:1075600093051000130101016FE00FB9130101FF32
:1075700023261100EF00001F1307100093070000DF
:10758000631AE5008320C100138507001301010180
:107590006780000017950100130545E3EFF0DFD287
:1075A0008320C10093072000138507001301010108
:1075B00067800000737004306F0000006780000077
:1075C000737004306F000000130101FD2324810259
:1075D0002322910223202103232E3101232C410158
:1075E000232611021309000017940100130404FB61
:1075F00097990100938989FB179A0100130ACAF928
:10760000930410000325040093050000EFA09FA33E
:10761000E30A05FE93060000130600009305C1006F
:10762000EFA08F80630695009797010023A007F8CD
:107630008327C100638427039797010023A807F6D7
:1076400083A70900E39097FC83270A00938717001C
:10765000179701002322F7F46FF0DFFA13091900DE
:107660006FF01FFE130101FF130600009305400099
:107670001305A0002326110023248100EF904FDA88
:10768000179401001304C4F12320A4001305A000E3
:10769000EFA01F83930705000325040093850700CF
:1076A00017970100232CF7EEEFA05F8E03248100D3
:1076B0008320C10093080000130800009307000016
:1076C0001307000093060000130600409795010081
:1076D000938505D417050000130545EF130101013B
:1076E0006FA0DFA4979701009387C7EA83A70700DD
:1076F00013072003938717006368F70017970100AB
:10770000232AF7E867800000130101FF9797010023
:10771000938707E92326110003A5070093060000BD
:107720001306000097950100938585E69797010061
:1077300023A207E6EF90DFBD93071000631EF5005C
:10774000979701009387C7E483A7070093871700E3
:1077500017970100232EF7E28320C10013010101D6
:107760006780000097970100938707E31797010050
:107770001307C7E183A70700032707006316F70075
:1077800017970100232407E217970100130707E268
:107790000325070017970100232AF7DE6780000002
:1077A000B305B500930705006386B70003C707005C
:1077B000631607003385A740678000009387170092
:1077C0006FF09FFE130101FB23229104232C410340
:1077D000232291032326110423248104232021053D
:1077E000232E3103232A5103232861032326710307
:1077F000232481032320A103232EB101930C050030
:10780000138A05009304000063DE05003305A040E1
:107810003337A000B305B040930C0500338AE54030
:107820009304F0FF63DA06003306C040B337C000AC
:10783000B306D040B386F640930A0600938906004B
:1078400013840C0013090A0063960628179B010095
:10785000130B4BA66370CA16B70701006372F614C8
:107860009307F00F63F4C70093098000B357360104
:10787000330BFB0083470B0013050002B38737016E
:10788000B309F540638C0900B3153A01B3D7FC0086
:10789000B31A360133E9B70033943C0113DB0A0114
:1078A00093050B0013050900EF00507C130A050037
:1078B00093050B00939B0A0113050900EF009076D6
:1078C00093DB0B019305050013850B00EF00D072CD
:1078D000131A0A0193570401B367FA0063FAA70069
:1078E000B387570163E6570163F4A700B3875701D5
:1078F0003389A74093050B0013050900EF001077AB
:10790000130A050093050B0013050900EF009071A1
:107910001314040193050500131A0A0113850B00C3
:1079200013540401EF00506D33648A00637AA4009D
:1079300033045401636654016374A4003304540196
:107940003304A4403354340193050000638A0400D7
:1079500033048040B3378000B305B040B385F540B1
:10796000130504008320C1040324810483244104FB
:10797000032901048329C103032A8103832A4103C4
:10798000032B0103832BC102032C8102832C4102B0
:10799000032D0102832DC101130101056780000041
:1079A000B707000193090001E362F6EC9309800137
:1079B0006FF0DFEB631A060093050000130510005B
:1079C000EF005066930A0500B707010063FAFA0E4C
:1079D0009307F00F63F4570193098000B3D73A017E
:1079E000330BFB0083470B001305000233095A4198
:1079F000B3873701B309F540E38209EAB39A3A0144
:107A0000335BFA00B3153A01B3D7FC0093DB0A01EC
:107A100033E9B70013050B0093850B00EF001065E9
:107A2000130A050093850B00139C0A0113050B0034
:107A3000EF00505F135C0C019305050013050C006B
:107A4000EF00905B131A0A0193570901B367FA001C
:107A500033943C0163FAA700B387570163E65701EB
:107A600063F4A700B3875701338BA74093850B00BE
:107A700013050B00EF00905F130A050093850B00C0
:107A800013050B00EF00105A9305050013050C00B9
:107A9000EF00905693160901131A0A0193D60601B6
:107AA000B366DA0063FAA600B386560163E65601B0
:107AB00063F4A600B38656013389A6406FF01FDE3B
:107AC000B707000193090001E3EAFAF09309800186
:107AD0006FF0DFF06376DA0093050A006FF01FE7BE
:107AE000B707010063FAF604930BF00F33B5DB0020
:107AF0001315350033D7A600978701009387877B3E
:107B0000B387E70083CB070093050002B38BAB007C
:107B1000338B7541631C0B0263E4460163EACC00BE
:107B20003384CC40B306DA4033B98C003389264124
:107B3000930509006FF09FE1B707000113050001ED
:107B4000E3EAF6FA130580016FF0DFFAB3966601F7
:107B5000335D7601336DDD00B35D7A01B3156A01E3
:107B600033DC7C0113540D01336CBC0013850D0014
:107B700093050400B3196601EF00504F930A050006
:107B80009305040013850D0033996C01931C0D01BE
:107B9000EF00504993DC0C01130A05009305050022
:107BA00013850C00EF005045939A0A0113570C01FE
:107BB00033E7EA00930D0A00637EA7003307A701AD
:107BC000930DFAFF6368A7016376A700930DEAFFA0
:107BD0003307A701330AA7409305040013050A00E1
:107BE000EF00D04893050400930A050013050A002E
:107BF000EF005043930505001304050013850C00A6
:107C0000EF00903F93150C01939A0A0193D505015B
:107C1000B3E5BA001307040063FEA500B385A50110
:107C20001307F4FF63E8A50163F6A5001307E4FF5B
:107C3000B385A501939D0D01B70C0100B3EDED00D7
:107C40001384FCFFB3F78D0033F48900338AA54019
:107C500013850700930504002326F10093DD0D0131
:107C6000EF00903993050400930A050013850D0079
:107C7000EF00903813DC090193050C002324A100C8
:107C800013850D00EF0050378327C10013040C004B
:107C900093050400130C050013850700EF00D03591
:107CA0008326810013D70A013305D5003307A700C7
:107CB0006374D700330C9C01B70701009387F7FF6B
:107CC000935507013377F70013170701B3F7FA004D
:107CD000B3858501B307F7006366BA00631EBA0077
:107CE000637CF90033863741B3B7C700B385A5413C
:107CF000B385F54093070600B307F9403339F9001F
:107D0000B305BA40B385254133947501B3D76701F4
:107D10003364F400B3D565016FF05FC3130101FD57
:107D200023229102232A51012326110223248102B6
:107D300023202103232E3101232C4101232861011B
:107D40002326710123248101232291012320A101F3
:107D5000930A050093840500639E06381304060009
:107D600093090500178901001309C95463F8C51266
:107D7000B7070100138B05006378F6101307F00FA7
:107D80003337C70013173700B357E6003309F9003C
:107D9000834609003387E60093060002B386E64077
:107DA000638C0600B394D40033D7EA003314D600B2
:107DB000336B9700B399DA00935A040193850A0054
:107DC00013050B00EF00902A1309050093850A00A4
:107DD000931B040113050B00EF00D02493DB0B0170
:107DE000930405009305050013850B00EF00D020D8
:107DF0001319090193D70901B367F900138A040025
:107E000063FEA700B3878700138AF4FF63E8870047
:107E100063F6A700138AE4FFB3878700B384A74003
:107E200093850A0013850400EF0050241309050010
:107E300093850A0013850400EF00D01E9399090171
:107E400093040500930505001319090113850B0020
:107E500093D90901EF00501AB36939011386040060
:107E600063FCA900B30934011386F4FF63E68900BB
:107E700063F4A9001386E4FF13140A013364C400F9
:107E8000130A00006F000013B70700011307000179
:107E9000E36CF6EE130780016FF01FEF138A060004
:107EA000631A06009305000013051000EF009017F9
:107EB00013040500B7070100637EF4129307F00F67
:107EC00063F48700130A8000B35744013309F900B3
:107ED000034709009306000233074701B386E640D3
:107EE00063940612B3848440130A1000135B0401E8
:107EF00093050B0013850400EF00501713090500CC
:107F000093050B0013850400931B0401EF009011EF
:107F100093DB0B01930405009305050013850B000B
:107F2000EF00900D1319090193D70901B367F90008
:107F3000938A040063FEA700B3878700938AF4FF47
:107F400063E8870063F6A700938AE4FFB38787009E
:107F5000B384A74093050B0013850400EF001011B4
:107F60001309050093050B0013850400EF00900B27
:107F7000939909019304050093050500131909015C
:107F800013850B0093D90901EF001007B36939017C
:107F90001386040063FCA900B30934011386F4FFBF
:107FA00063E6890063F4A9001386E4FF13940A01D1
:107FB0003364C4001305040093050A008320C10242
:107FC0000324810283244102032901028329C10180
:107FD000032A8101832A4101032B0101832BC10064
:107FE000032C8100832C4100032D010013010103A8
:107FF00067800000B7070001130A0001E366F4EC94
:10800000130A80016FF05FEC3314D40033DAE4001C
:10801000B399DA0033D7EA00935A0401B394D40039
:1080200093850A0013050A00336B9700EF001004D4
:108030001309050093850A0013050A00931B040128
:10804000EF00407E93DB0B019304050093050500D0
:1080500013850B00EF00407A1319090113570B0128
:108060003367E900138A0400637EA70033078700A3
:10807000138AF4FF636887006376A700138AE4FF1E
:1080800033078700B304A74093850A0013850400D3
:10809000EF00C07D1309050093850A0013850400D5
:1080A000EF004078930405009305050013850B004D
:1080B000EF00807413170B011357070113190901FF
:1080C000B367E9001387040063FEA700B387870046
:1080D0001387F4FF63E8870063F6A7001387E4FFC4
:1080E000B3878700131A0A01B384A740336AEA00F2
:1080F0006FF0DFDF63ECD51EB707010063F4F60411
:108100001307F00FB335D7009395350033D7B6007A
:10811000978701009387071AB387E70003C7070013
:10812000130A00023307B700330AEA4063160A0253
:1081300013041000E3E096E833B6CA0013441600B7
:108140006FF05FE7B707000193050001E3E0F6FC7D
:10815000930580016FF09FFBB35CE600B396460188
:10816000B3ECDC0033D4E40093DB0C01B39744019F
:1081700033D7EA0093850B0013050400336BF70037
:10818000B3194601EF00806E1309050093850B00BB
:1081900013050400139C0C01EF00C068135C0C0174
:1081A000930405009305050013050C00EF00C0645F
:1081B0001319090113570B013367E90013840400F5
:1081C000637EA700330797011384F4FF6368970168
:1081D0006376A7001384E4FF33079701B304A74035
:1081E00093850B0013850400EF0040681309050018
:1081F00093850B0013850400EF00C0629304050013
:108200009305050013050C00EF00005F93170B01A9
:108210001319090193D70701B367F9001386040006
:1082200063FEA700B38797011386F4FF63E8970105
:1082300063F6A7001386E4FFB387970113140401C4
:10824000B70B01003364C4001389FBFF337D2401A5
:1082500033F92901B384A7409305090013050D00E4
:10826000EF008059935C040193050900130B05008E
:1082700013850C00EF00405893D90901130C050039
:108280009385090013850C00EF00005713090500C2
:108290009385090013050D00EF0000563305850195
:1082A00093570B013385A700637485013309790166
:1082B00093570501B387270163E6F402E392F4BC08
:1082C000B70701009387F7FF3375F5001315050114
:1082D000337BFB0033964A0133056501130A000026
:1082E000E37AA6CC1304F4FF6FF09FB9130A0000E1
:1082F000130400006FF01FCC130101FB2324810441
:1083000023229104232E31032322910323261104D7
:1083100023202105232C4103232A51032328610311
:1083200023267103232481032320A103232EB101DB
:10833000930C050093890500130405009384050040
:10834000639E062613090600138A0600978A010019
:10835000938A4AF663F4C514B70701006376F612F0
:108360009307F00F63F4C700130A8000B357460168
:10837000B38AFA0003C70A00130500023307470156
:10838000330AE540630C0A00B395490133D7EC008A
:1083900033194601B364B70033944C01935A090171
:1083A00093850A0013850400EF00404C93090500F3
:1083B00093850A00131B090113850400EF00804612
:1083C000135B0B019305050013050B00EF00C04282
:1083D0009399090193570401B3E7F90063FAA700E1
:1083E000B387270163E6270163F4A700B38727015A
:1083F000B384A74093850A0013850400EF0000476B
:108400009309050093850A0013850400EF0080415D
:1084100013140401930505009399090113050B003A
:1084200013540401EF00403D33E48900637AA40053
:1084300033042401636624016374A400330424011B
:108440003304A44033554401930500008320C10444
:108450000324810483244104032901048329C103E3
:10846000032A8103832A4103032B0103832BC102C7
:10847000032C8102832C4102032D0102832DC101B3
:108480001301010567800000B7070001130A00010E
:10849000E36EF6EC130A80016FF05FED631A0600DD
:1084A0009305000013051000EF00C0371309050005
:1084B000B7070100637AF90E9307F00F63F4270101
:1084C000130A8000B3574901B38AFA0003C70A00B0
:1084D00013050002B384294133074701330AE540FD
:1084E000E30E0AEA33194901B3DAE900B395490109
:1084F00033D7EC0093540901336BB70013850A009E
:1085000093850400EF0080369309050093850400ED
:10851000931B090113850A00EF00C03093DB0B01A8
:108520009305050013850B00EF00002D93990901B9
:1085300093570B01B3E7F90033944C0163FAA7009A
:10854000B387270163E6270163F4A700B3872701F8
:10855000B38AA7409385040013850A00EF00003119
:10856000930905009385040013850A00EF00802B12
:108570009305050013850B00EF00002893150B01F0
:108580009399090193D50501B3E5B90063FAA500F4
:10859000B385250163E6250163F4A500B3852501B4
:1085A000B384A5406FF09FDFB7070001130A0001F5
:1085B000E36AF9F0130A80016FF0DFF0E3E8D5E831
:1085C000B707010063FCF604930BF00F33B5DB0033
:1085D0001315350033D7A60097870100938787CD01
:1085E000B387E70083CB070093050002B38BAB0092
:1085F000338B7541631E0B0263E4360163EACC00E2
:108600003384CC40B386D94033B58C00B384A640C4
:1086100013050400938504006FF05FE3B7070001C2
:1086200013050001E3E8F6FA130580016FF09FFAE5
:10863000B3966601335D7601336DDD0033D4790185
:10864000B395690133DC7C0193540D01336CBC009C
:108650001305040093850400B31A6601EF0000219E
:10866000130A0500938504001305040033996C0177
:10867000931C0D01EF00001B93DC0C01130405009B
:108680009305050013850C00EF000017131A0A016B
:1086900013570C013367EA00130A0400637EA70036
:1086A0003307A701130AF4FF6368A7016376A700E5
:1086B000130AE4FF3307A701B309A7409385040019
:1086C00013850900EF00801A938504001304050048
:1086D00013850900EF0000159305050093040500BC
:1086E00013850C00EF00401193150C0113140401C5
:1086F00093D50501B365B4001387040063FEA5009C
:10870000B385A5011387F4FF63E8A50163F6A5000F
:108710001387E4FFB385A501131A0A01B70C010002
:10872000336AEA001384FCFFB3778A0033F48A00CB
:10873000B384A54013850700930504002326F100A8
:10874000135A0A01EF00400B93090500930504003A
:1087500013050A00EF00400A13DC0A01930D05001F
:1087600093050C0013050A00EF0000098327C100E0
:10877000130A050093050C0013850700EF00C007DE
:108780003305B50113D709013307A7006374B70197
:10879000330A9A01B70701009387F7FF9355070142
:1087A0003377F70013170701B3F7F900B3854501D5
:1087B000B307F70063E6B400639EB400637CF9007E
:1087C00033865741B3B7C700B385A541B385F5409C
:1087D00093070600B307F9403339F900B385B44075
:1087E000B385254133947501B3D767013365F40030
:1087F000B3D565016FF09FC5130605001305000092
:1088000093F61500638406003305C50093D5150063
:1088100013161600E39605FE678000006340050608
:1088200063C6050613860500930505001305F0FFD2
:10883000630C060293061000637AB6006358C0000A
:108840001316160093961600E36AB6FE1305000091
:1088500063E6C500B385C5403365D50093D61600E1
:1088600013561600E39606FE678000009382000010
:10887000EFF05FFB13850500678002003305A04021
:1088800063D80500B305B0406FF0DFF9B305B04021
:1088900093820000EFF01FF93305A04067800200CB
:1088A0009382000063CA0500634C0500EFF09FF758
:1088B0001385050067800200B305B040E35805FE4C
:1088C0003305A040EFF01FF63305B040678002008B
:1088D00097870100938747C883A607001787010081
:1088E000130747C60327070023A2A600637EE500FF
:1088F000178701001307C7C50325070083A50700D5
:10890000938545006F701FE8130101FF2324810048
:1089100023261100178701001307C7C3130405009E
:108920000325070083A5070093854500EF709FE5A9
:1089300097870100938747BF83A707006376F400FA
:108940009787010023A287BE8320C10003248100F2
:108950001301010167800000978701009387C7BF5B
:1089600003A7070083A60700832747049387F7FF21
:108970002322F70483A7460463940700736004303E
:1089800067800000130101FE232C8100232A91003F
:1089900013040500938405002328210123263101B7
:1089A0002324410123225101232E1100EFA04FE483
:1089B0008327040003290401B7090001B3E59700E8
:1089C000930AC4002320B400930400009389F9FFA4
:1089D000370A00020327040063822A0503260900E0
:1089E00013050900B3654701B376360193175600A6
:1089F00033F7E6000329490063C607006316070042
:108A00006FF05FFDE398E6FC9317760063D40700F0
:108A1000B3E4D400EFB01FA66FF0DFFB93C4F4FF04
:108A2000B3F4E40023209400EFA01F90032504007A
:108A30008320C10103248101832441010329010111
:108A40008329C100032A8100832A41001301010206
:108A500067800000130101FF2326110023248100F9
:108A6000EFE01FAB17F7FFFF1307479A93060000CD
:108A7000130610009305400617850100130585981D
:108A8000EFC09FD56302050213040500EFA0CFD706
:108A9000130605001307000093060000930510005D
:108AA00013050400EFC05FE5EFA0CFA18320C10054
:108AB00003248100130500001301010167800000F9
:02000004800278
:10000000F467FEFF6469FEFF0068FEFF6469FEFF9F
:100010006469FEFF6469FEFF6469FEFF2868FEFFF5
:100020006469FEFF6469FEFF5068FEFF6068FEFFC2
:100030006469FEFF7868FEFF8868FEFF8868FEFF3F
:100040008868FEFF8868FEFF8868FEFF8868FEFFFC
:100050008868FEFF8868FEFF8868FEFF6469FEFF0F
:100060006469FEFF6469FEFF6469FEFF6469FEFF68
:100070006469FEFF6469FEFF6469FEFF6469FEFF58
:100080006469FEFF6469FEFF6469FEFF6469FEFF48
:100090006469FEFF6469FEFF6469FEFF6469FEFF38
:1000A0006469FEFF6469FEFF6469FEFF6469FEFF28
:1000B0006469FEFF6469FEFF6469FEFF6469FEFF18
:1000C0006469FEFF6469FEFF6469FEFF6469FEFF08
:1000D0006469FEFF6469FEFF6469FEFF6469FEFFF8
:1000E0006469FEFF6469FEFF6469FEFF6469FEFFE8
:1000F0006469FEFF6469FEFF6469FEFF6469FEFFD8
:10010000CC68FEFFF468FEFF6469FEFF6469FEFFD1
:100110006469FEFF6469FEFF6469FEFF6469FEFFB7
:100120006469FEFF5469FEFF6469FEFF6469FEFFB7
:100130000466FEFF0C67FEFF6469FEFF6469FEFF54
:100140005C67FEFF6469FEFFD467FEFF6469FEFF23
:100150006469FEFF1C68FEFFC06DFEFF2C6EFEFF93
:10016000CC6DFEFF2C6EFEFF2C6EFEFF2C6EFEFF94
:100170002C6EFEFF646CFEFF2C6EFEFF2C6EFEFFED
:100180008C6CFEFF9C6CFEFF2C6EFEFFB46CFEFFC1
:10019000C46CFEFFC46CFEFFC46CFEFFC46CFEFFAB
:1001A000C46CFEFFC46CFEFFC46CFEFFC46CFEFF9B
:1001B000C46CFEFF2C6EFEFF2C6EFEFF2C6EFEFF4D
:1001C0002C6EFEFF2C6EFEFF2C6EFEFF2C6EFEFFD3
:1001D0002C6EFEFF2C6EFEFF2C6EFEFF2C6EFEFFC3
:1001E0002C6EFEFF2C6EFEFF2C6EFEFF2C6EFEFFB3
:1001F0002C6EFEFF2C6EFEFF2C6EFEFF2C6EFEFFA3
:100200002C6EFEFF2C6EFEFF2C6EFEFF2C6EFEFF92
:100210002C6EFEFF2C6EFEFF2C6EFEFF2C6EFEFF82
:100220002C6EFEFF2C6EFEFF2C6EFEFF2C6EFEFF72
:100230002C6EFEFF2C6EFEFF2C6EFEFF2C6EFEFF62
:100240002C6EFEFF2C6EFEFF2C6EFEFF2C6EFEFF52
:100250002C6EFEFF2C6EFEFF086DFEFF446DFEFF50
:100260002C6EFEFF2C6EFEFF2C6EFEFF2C6EFEFF32
:100270002C6EFEFF2C6EFEFF2C6EFEFFB06DFEFF9F
:100280002C6EFEFF2C6EFEFF386AFEFF8C6BFEFFAD
:100290002C6EFEFF2C6EFEFF1C6CFEFF2C6EFEFF14
:1002A000486CFEFF2C6EFEFF2C6EFEFF206EFEFFE4
:1002B000000102020303030304040404040404040D
:1002C00005050505050505050505050505050505DE
:1002D00006060606060606060606060606060606BE
:1002E00006060606060606060606060606060606AE
:1002F000070707070707070707070707070707078E
:10030000070707070707070707070707070707077D
:10031000070707070707070707070707070707076D
:10032000070707070707070707070707070707075D
:10033000080808080808080808080808080808083D
:10034000080808080808080808080808080808082D
:10035000080808080808080808080808080808081D
:10036000080808080808080808080808080808080D
:1003700008080808080808080808080808080808FD
:1003800008080808080808080808080808080808ED
:1003900008080808080808080808080808080808DD
:1003A00008080808080808080808080808080808CD
:1003B000546D725100000000546D7220537663003A
:1003C000286E756C6C2900004572726F7220696E20
:1003D00020787878207461736B73200D0A00000018
:1003E0006D69616F750A00006D69616F75320A0091
:1003F00068756E6772790A0054696D657232000023
:10040000436865636B54696D657200005365745091
:040410006F6C6C00A1
:100414001000000000000000017A5200017C01017C
:100424001B0D020050000000180000009473FEFF32
:100434005805000000440E507489039406990B81FA
:1004440001880292049305950796089709980A9AD9
:100454000C9B0D036C010AC144C844C944D244D363
:1004640044D444D544D644D744D844D944DA44DBAC
:10047400440E00440B0000004C0000006C0000001F
:100484009878FEFFDC05000000440E307089039567
:1004940007810188029204930594069608970998A7
:1004A4000A990B9A0C0370020AC144C844C944D285
:1004B40044D344D444D544D644D744D844D944DA64
:1004C400440E00440B00000050000000BC0000007B
:1004D400247EFEFF0005000000440E50748802894B
:1004E400039305990B810192049406950796089746
:1004F40009980A9A0C9B0D0320010AC144C844C9F7
:1005040044D244D344D444D544D644D744D844D91B
:0C05140044DA44DB440E00440B000000FD
:0C05A000FC8F01000900000001000000B9
:040000058000004037
:00000001FF
